:10C00000E80C01205DE20000E92501008DE200005E
:10C010008DE200008DE200008DE200008DE2000064
:10C0200000000000000000000000000031E00000FF
:10C030008DE2000000000000D9DF0000CD250100E6
:10C040001DE200001DE200001DE200001DE20000F4
:10C050001DE200001DE200001DE200001DE20000E4
:10C060001DE200001DE200001DE200001DE20000D4
:10C070001DE200001DE200001DE200001DE20000C4
:10C080001DE200001DE200001DE200001DE20000B4
:10C090001DE200001DE200001DE200001DE20000A4
:10C0A0001DE200001DE200001DE200001DE2000094
:10C0B0001DE200001DE200001DE200001DE2000084
:10C0C0001DE200001DE200001DE200001DE2000074
:10C0D0001DE200001DE200001DE200001DE2000064
:10C0E0001DE200001DE200001DE200001DE2000054
:10C0F0001DE200001DE200001DE200001DE2000044
:10C100001DE200001DE200001DE200001DE2000033
:10C110001DE200001DE200001DE200001DE2000023
:10C120001DE200001DE200001DE200001DE2000013
:10C130001DE200001DE200001DE200001DE2000003
:10C140001DE20000000000000000000000000000F0
:10C1500000000000000000000000000000000000DF
:10C1600000000000000000000000000000000000CF
:10C1700000000000000000000000000000000000BF
:10C1800000000000000000000000000000000000AF
:10C19000000000000000000000000000000000009F
:10C1A000000000000000000000000000000000008F
:10C1B000000000000000000000000000000000007F
:10C1C000000000000000000000000000000000006F
:10C1D000000000000000000000000000000000005F
:10C1E000000000000000000000000000000000004F
:10C1F000000000000000000000000000000000003F
:10C20000DEE61E284CBBCE8F025B00003C00000027
:10C21000247F00000100000000C0000000C00000FA
:10C22000FFFF02910000000000000000000000007D
:0CC2300000000000000000000000000002
:10C23C0053B94AB9002908BF00281CBF4FF0FF3181
:10C24C004FF0FF3000F070B9ADF1080C6DE904CE81
:10C25C0000F006F8DDF804E0DDE9022304B07047D5
:10C26C002DE9F047089E0D4604468A46002B7FD1E7
:10C27C008A42174641D9B2FA82F24AB1C2F1200180
:10C28C0005FA02F39740944020FA01F141EA030ABF
:10C29C004FEA17484FEA144C1FFA87F9BAFBF8FE1D
:10C2AC0008FB1EA30EFB09F14CEA0343994206D985
:10C2BC00FB1802D2994200F224810EF1FF3E591A6A
:10C2CC00A3B2B1FBF8F008FB101100FB09F943EA2B
:10C2DC000144A14505D93C1902D2A14500F20E81B9
:10C2EC000138A4EB090440EA0E4000211EB1D440F1
:10C2FC000023C6E90043BDE8F08702B9FFDEB2FABD
:10C30C0082F2002A4FD1CB1B4FEA174E1FFA87F847
:10C31C000121250CB3FBFEFC0EFB1C302B4608FB4D
:10C32C000CF945EA0045A9450AD97D192CBF012312
:10C33C000023A94502D9002B00F0D9800CF1FF3C59
:10C34C00A5EB0905A3B2B5FBFEF00EFB105508FBDF
:10C35C0000F843EA0544A04505D93C1902D2A04592
:10C36C0000F2C9800138A4EB080440EA0C40BDE798
:10C37C008B4208D9002E00F0B1800021C6E90005DF
:10C38C000846BDE8F087B3FA83F1002946D1AB42E9
:10C39C00C0F0A780824240F2A4800846002EAAD0AA
:10C3AC00C6E9004AA7E7C2F12000974001FA02F360
:10C3BC004FEA174EC14024FA00F51FFA87F8944053
:10C3CC001D43B1FBFEF02B0C0EFB101100FB08FC07
:10C3DC0043EA01439C4509D9FB182CBF01210021DC
:10C3EC009C4502D9002900F095800138A3EB0C0381
:10C3FC00ADB2B3FBFEF10EFB113301FB08FC45EAB9
:10C40C000345AC4505D97D1902D2AC4500F28980B3
:10C41C000139A5EB0C0341EA00417AE7C1F1200494
:10C42C008B4002FA01F705FA01FCE24020FA04F80D
:10C43C00E54000FA01FE134348EA0C024FEA1348A8
:10C44C004FEA124C1FFA83F9B5FBF8FA08FB1A55A0
:10C45C000AFB09F04CEA054C60450AD913EB0C0CAD
:10C46C002CBF01250025604501D9002D55D00AF1BE
:10C47C00FF3AACEB000C92B2BCFBF8F008FB10CC12
:10C48C0000FB09F942EA0C4CE14505D913EB0C0C05
:10C49C0001D2E1453BD8013840EA0A40ACEB090C2B
:10C4AC00A0FB0789CC4545464A4602D306D1C64572
:10C4BC0004D20138B8EB070569EB03022EB3BEEBCF
:10C4CC0005036CEB020C23FA01F20CFA04F42CFABF
:10C4DC0001F300211443C6E900430CE73146304612
:10C4EC0009E7841A65EB030301209A4656E7ACF181
:10C4FC00020C3D4424E702383C4434E702383C4407
:10C50C00EFE6AEF1020E3B44D9E63146F3E60238D3
:10C51C009C44C1E702383B4468E7AAF1020A9C44F8
:10C52C00A7E702393D4474E7704700BF2DE9F04F8F
:10C53C002B4887B005F083FA2A4804F0E1F9054648
:10C54C0030B92849284805F07AFA07B0BDE8F08FD1
:10C55C0000240A34E4B2FE2C28BF0024AB681D2151
:10C56C0028465B6804AA9847039078BBDDE9046B06
:10C57C00FD23A6FB038903FB0B991C4A00234046B1
:10C58C004946FFF755FE4FF0FF32194B82464B459B
:10C59C0008BF42451AD3A4FB066704FB0B770023A4
:10C5AC00124A30463946FFF743FE4FF0FF31104A2E
:10C5BC000346BA4208BFB14208D30399AA68009156
:10C5CC0016681D2152462846B04710B1094805F09F
:10C5DC0036FA002141F69A1004F0A2FEB9E700BF2A
:10C5EC00EC3201000B3301001133010040420F000B
:10C5FC003F420F00A43301000B6801330B60014B69
:10C60C001B68184700000120014B1860704700BFE1
:10C61C000000012007B50B4600210246019103489A
:10C62C0001A900F0FFF803B05DF804FB05C600009B
:10C63C0030B5002585B0CDE90101044601A90548B6
:10C64C00039500F0EFF8DDE902309842B8BF2554AD
:10C65C0005B030BD251A01002DE9F84FB0F818903F
:10C66C00044619F0080893460DD001290CBF49F077
:10C67C00100949F02009A0F818908BF31188BFF32A
:10C68C006F8FBDE8F88F09F00709022907D1204602
:10C69C0005F0EFF90028F0D00128238B50D1676901
:10C6AC00218B002F15DA256821F00701C4E90088D9
:10C6BC0041F0010121830026218B01F0070ACA45B4
:10C6CC0002D0A368002B5CD10DB9002E74D00023CE
:10C6DC0058E001F007035A1F012A20D821F0070166
:10C6EC00062B256889B2C4E900880CD1002D2B4695
:10C6FC0038BF00232BB1628B1B6801326283002B85
:10C70C00F8D141F002012046218305F0B2F906462A
:10C71C000028D1D0238B43F020032383CBE7042BB9
:10C72C000CD121F0070189B22046218305F0A1F933
:10C73C0005460028BFD041F0200121830025BAE72F
:10C74C00032809D1226923F00703166843F0060376
:10C75C00002523832F46AFE7042806D1226923F056
:10C76C000703566843F00403F2E7052806D1226953
:10C77C0023F00703966843F00503E9E700252E46EE
:10C78C00E8E7012341F0080121838BF31188BFF303
:10C79C006F8F03BB002D33D116B120462049B04713
:10C7AC004FF02003EFF3118B83F31188BFF36F8FDE
:10C7BC00238B23F008032383238BDA0628D501214E
:10C7CC0023F010032383B4F8189009F0070900290B
:10C7DC007FF45BAF51E7A1680029DBD00B68002B1D
:10C7EC0038BF0023994652463B462046D1F804B048
:10C7FC00D847B9F1000FCDD04946D9F80030EEE753
:10C80C0029463B46524620462D6805F04EF9C1E7B5
:10C81C0013F020011EBF23F0200302212383D2E753
:10C82C00E31A01002DE9F04F8B4692461C46002579
:10C83C0091B002909AF8000008B928465EE32528CA
:10C84C000AF1010707D05946029B98470028C0F20D
:10C85C005583013510E2182200210AA805F051FF7A
:10C86C009AF80130252B78D000229446164696462D
:10C87C001046394617F8013B2B2B00F09D8000F237
:10C88C009480202B00F09B80232B00F09A8028B101
:10C89C009DF8300040F004008DF83000BEF1000F20
:10C8AC0005D09DF8300040F008008DF830002EB116
:10C8BC009DF8300040F010008DF83000BCF1000FF6
:10C8CC0005D09DF8300040F020008DF830002AB1E2
:10C8DC009DF8302042F040028DF830209DF8302039
:10C8EC0002F04400442803D16FF386128DF83020F7
:10C8FC009DF830202A2B42F080028DF830207BD11D
:10C90C009DF831204B1C42F001028DF831201A7831
:10C91C002E2A0CBF012100219DF8312061F3410228
:10C92C008DF8312074D15A782A2A6AD000210A262F
:10C93C000133184610F8012BA2F13007092F40F2F1
:10C94C008E809DF830200E91C2F3400040EAD171E8
:10C95C0061F341028DF830205AE00AF102078DF89C
:10C96C0033309DF83130D90740F1498154F8049B9C
:10C97C00B9F1000F07DA9DF83020C9F1000942F037
:10C98C0004028DF830205A0740F1428154F8048B90
:10C99C00B8F1000F80F241819DF831306FF3410303
:10C9AC008DF831304FF0FF3837E12D2B0CD0302B78
:10C9BC007FF46DAF01225CE74FF0010E59E70126C1
:10C9CC0057E74FF0010C54E7012052E733460CFBBC
:10C9DC000202303A1E4616F8010BA0F13007092F5F
:10C9EC00F4D9994293D09DF830100D92D20F62F386
:10C9FC0041018DF830108AE70B4600224FF00A0CEB
:10CA0C00E8E79DF83120023342F004028DF8312022
:10CA1C001F4617F8012B6C2A41D025D8682A2BD039
:10CA2C006A2A46D04C2A4CD01F4617F8012B9DF889
:10CA3C003130782A8DF8332000F2D980572A4DD81E
:10CA4C00412A03D0453A022A00F2D18004229DF8F3
:10CA5C00323062F302038DF8323001239EE006FB84
:10CA6C0001210346303964E7742A26D07A2ADBD1B7
:10CA7C0006229DF831300DE05A78682A9DF8312055
:10CA8C0006D1012161F3C6028DF831209F1CCCE741
:10CA9C001346022262F3C6038DF83130C5E75A788B
:10CAAC006C2A9DF8312001D10421EBE713460322B7
:10CABC00F0E705229DF83130ECE707229DF8313084
:10CACC00E8E7BDF8303023F4F04323F0020343F4DD
:10CADC00804343F00203ADF83030A6E7A2F15801D1
:10CAEC00202900F2848001A050F821F0BDCB000079
:10CAFC00FBCB0000FBCB0000FBCB0000FBCB000012
:10CB0C00FBCB0000FBCB0000FBCB0000FBCB000001
:10CB1C0059CA0000FBCB0000BDCB00007DCB000050
:10CB2C0059CA000059CA000059CA0000FBCB0000CA
:10CB3C007DCB0000FBCB0000FBCB0000FBCB00004F
:10CB4C00FBCB0000C5CB0000BDCB0000E1CB00004F
:10CB5C00FBCB0000FBCB0000E1CB0000FBCB0000CB
:10CB6C00BDCB0000FBCB0000FBCB0000BDCB00001D
:10CB7C0001209DF8321003F0780360F30201402B82
:10CB8C008DF8321002BF9DF8301041F001018DF884
:10CB9C003010632A31D1003B18BF01239DF830209F
:10CBAC00C2F340010B4363F341028DF83020D8E609
:10CBBC0002209DF83210DEE703219DF8322003F0AD
:10CBCC007803A3F1400061F3020243428DF8322056
:10CBDC004341E3E703219DF8322013F0780F61F312
:10CBEC00020214BF012300238DF83220D6E79DF8F2
:10CBFC00303043F001038DF830300023CEE79DF93F
:10CC0C003020002AACBF4FF0FF39DDF83490BAE683
:10CC1C009B077FF5C7AEDDF838800023CDE90D33D7
:10CC2C009DF832309DF8312003F00703012BC2F33D
:10CC3C00C30236D1D31E042B20D8DFE803F0030740
:10CC4C00071F1F0054F8040BC11704E0073424F02D
:10CC5C000704F4E80201CDE90A019DF8303013F025
:10CC6C00030654D03B4652465946029805F0DDF86F
:10CC7C000028C0F243810544BA46DBE554F8040BA6
:10CC8C00012A4FEAE071CDE90A0105D19DF828305F
:10CC9C000A9300230B93E0E7022ADED1BDF92800AA
:10CCAC00D2E7022B23D1D31E042B13D8DFE803F0D9
:10CCBC00030A0A12120000212068231D0A900B910E
:10CCCC001C46CAE7073424F00703F3E80201CDE958
:10CCDC000A01F5E754F8043B012A0A934FF00003CC
:10CCEC000B93D3D0022AB8D1BDF82830D0E7042B4F
:10CCFC0007D1073424F00704F4E80201CDE90A0156
:10CD0C00ABE7032B04BF54F8043B0A93A5E79DF84B
:10CD1C0033007828B0D8622822D825283FF493AD68
:10CD2C005828A9D1DDE90A010DF1260300930CAABC
:10CD3C0004AB05F02FF88246B8F1000F0DF1260078
:10CD4C000CDB9DF83020A0EB0A036FF3861298459C
:10CD5C008DF8302002D9A8EB03030D9380463DE0FB
:10CD6C006338152888D801A151F820F0F9CD0000BE
:10CD7C005DCE000085CC000085CC000085CC000089
:10CD8C0085CC00005DCE000085CC000085CC000079
:10CD9C0085CC000085CC0000BBCE000089CE000005
:10CDAC008DCE000085CC000085CC0000D1CD0000DC
:10CDBC0085CC000089CE000085CC000085CC00001D
:10CDCC0089CE0000B8F1000FDDF828A00ADB41463F
:10CDDC00504605F046FC00260AEB0008BAF1000F9D
:10CDEC000CD149E7504605F035FCF4E700260A9BC8
:10CDFC000DF111088DF810300DF1100AA8EB0A0393
:10CE0C0006B101339DF83220D0066BD502335206A1
:10CE1C000D9948BF0E9A0B4448BF9B18B9F1000FEF
:10CE2C0079DD9DF83020A9EB0309C2F3800303934D
:10CE3C00530770D4500664D546B159463046029B10
:10CE4C00984700285ADB039B01351E46302359E0D6
:10CE5C001E0711D413F0100618BF2026DDE90A2393
:10CE6C00002A73F10001BFF65DAF524263EB43033E
:10CE7C002D26CDE90A2355E72B26EFE7002651E7AF
:10CE8C000A9848B30DF126030093002104AB0CAAB9
:10CE9C0004F080FFBDF83230824603F0EF0343F418
:10CEAC00F04343F010030026ADF8323044E70A9B00
:10CEBC00072A3FF6E1AEDFE802F00D04060D080884
:10CECC000D0D1D70D8E61D80D6E62846E917C3E97E
:10CEDC000001D1E61D60CFE6DFF8C4800646A8F15C
:10CEEC00050A8BE7110748BF013390E718460393F7
:10CEFC005946029B98470028039B04DA11B0BDE801
:10CF0C00F08F20234D444A46002AA5EB090109F174
:10CF1C00FF39EBDC0D4636B159463046029B98473B
:10CF2C000028EBDB01359DF83230D90601D41A0705
:10CF3C0006D559463020029B98470028DEDB013588
:10CF4C009DF83230DB0607D559469DF83300029B1D
:10CF5C0098470028D2DB01350D9E2E44731B002B05
:10CF6C0016DC434652465946029804F05EFF0028F0
:10CF7C00C4DB0544A944A9EB0503002B7FF77CAE69
:10CF8C0059462020029B98470028B7DB0135F2E771
:10CF9C0059463020029B98470028AFDB0135DDE76E
:10CFAC00403301004FF02002EFF3118382F311881C
:10CFBC00BFF36F8F0121044AC2F8401583F3118827
:10CFCC00BFF36F8F002070470090034020B1034BDC
:10CFDC00800143F001031847704700BFB0300100D7
:10CFEC0030B5002289B00F490F4805F06DFE0022C4
:10CFFC0000230024CDE906230E230C4DCDE9033488
:10D00C004FF440722846CDE90144094B094900947C
:10D01C0004F028FA0849284605F00DFE204609B010
:10D02C0030BD00BF49D00000D80101201002012002
:10D03C0031D40000E805012045330100014804F01B
:10D04C0097B900BFC401012008B500F049FA09489E
:10D05C0004F004FF042328220749084805F0FAFCD1
:10D06C00074B084A4FF400401A60BDE8084000F036
:10D07C007FBC00BFA403012028160120AC030120B3
:10D08C0004000120A71E0100F8B500250C4BD3E8C5
:10D09C00EF7FC3E8E25F002AF9D10A4C0A4E361B37
:10D0AC003611B54200DBF8BD63685B792BB12368A0
:10D0BC00DB6813B139462046984701351034F0E748
:10D0CC009C0301205C3001006C300100044BD3E860
:10D0DC00EF2F0132C3E8E12F0029F8D1704700BFD0
:10D0EC009C030120044A054B9B1AB1EBD30F34BFB0
:10D0FC0052F8310000207047EC2F01005C30010029
:10D10C00094B4268C31A1B11013310B5137101226C
:10D11C004368064C5A712278196012B9044804F01D
:10D12C0027F90123237010BD5C300100DC050120C0
:10D13C00C401012070B50F4BD3E8EF5F6A1CC3E844
:10D14C00E12F0029F8D12DB90B4C0C4E361B3611A2
:10D15C00B54200DB70BD237B43B123685B6903B12F
:10D16C009847042200212046FFF7CAFF01351034EE
:10D17C00EEE700BFA00301205C3001006C30010021
:10D18C00144B37B59842044602D3134B98421CD328
:10D19C0000220023114801A903F034FD0546B8B95B
:10D1AC000122019BD3E8EF1FC3E8E02F0028F9D13F
:10D1BC00019821461F22043005F039FA7E23019C88
:10D1CC0084F8233084F824500434204603B030BD56
:10D1DC00034CFAE74C2D0100503D0100AC0301203B
:10D1EC004D33010048B1054B984205D3A03398420A
:10D1FC002CBF00200120704700207047281601200A
:10D20C002DE9F04F4A4B04461B7885B003B940B367
:10D21C004FF02003EFF3118683F31188BFF36F8F68
:10D22C00444804F02BFE054686F31188BFF36F8F3C
:10D23C0058B1414BD3E8EF2F013AC3E8E12F002955
:10D24C00F8D194B1284604F02EFF24B93B4B1B684F
:10D25C000BB1FFF719FF374804F00EFE041E18BF80
:10D26C000124204605B0BDE8F08F354B1B78CBB9B7
:10D27C002B7ADB0716D404F025FF8046284604F0F1
:10D28C00F0FE0146404604F00CFE06462D4F2E4B98
:10D29C00DFF8D0B0DB1BDB0803932C4BDB1B4FEA16
:10D2AC00D30A36B92A4E2B4F4FF00008BF1B3F1143
:10D2BC003AE0B6FA86F1C1F11F094946284604F056
:10D2CC00D3FE254B0146984202D3244B98421AD3E5
:10D2DC000846FFF787FF0246A8B9214B994212D0A6
:10D2EC006B890399C3F389138B4238BF57F83320EA
:10D2FC004FEA8A1343F00103ADF800304946434628
:10D30C00584604F028FE012101FA09F126EA01062B
:10D31C00C7E773685B7923B13368294630461B68CD
:10D32C00984708F101081036B845F2DB8AE700BFD0
:10D33C00DC050120A4030120980301209C0301209B
:10D34C00DD050120EC2F01005C30010014300100E0
:10D35C005C3001006C3001004C2D0100503D01008F
:10D36C004D33010067330100274B73B51B684181B6
:10D37C0004469847254DE060D5E8EF3F0133C5E8FA
:10D38C00E23F002AF8D14FF02003EFF3118683F32C
:10D39C001188BFF36F8F1E48214604F063FD86F39E
:10D3AC001188BFF36F8F1B4B1B7883B14FF0200399
:10D3BC00EFF3118483F31188BFF36F8F0020FFF715
:10D3CC001FFF84F31188BFF36F8F02B070BD124A38
:10D3DC002B681268002AF8D0012B0AD100220023F6
:10D3EC000E48CDE900234FF40042002304F086FAE6
:10D3FC00EBE70A2BE9D1094805F072FC084802B0AA
:10D40C00BDE8704003F0B4BF040001209803012074
:10D41C00A4030120DD050120C8030120D80101204F
:10D42C00C401012010B5FFF785FE03F09BFF0C4BE8
:10D43C00186030B10B4B1B68092B02DD0A4803F056
:10D44C0097FF094C0020FFF7DBFE0028FAD14FF0C4
:10D45C00FF324FF0FF33204603F0AAFFF2E700BF84
:10D46C00C803012098030120C4010120F8B50E4F18
:10D47C003D7875B9FFF75EFE0C4C0D4E361B361120
:10D48C00B54207DB0020FFF7BBFE0028FAD10123D1
:10D49C003B70F8BD63685B791BB1236820461B6940
:10D4AC00984701351034EBE7DD0501205C300100B5
:10D4BC006C30010007B504380190D0E8EF3F5A1EDC
:10D4CC00C0E8E12F0029F8D1012B03D1034801A9B1
:10D4DC0003F0CAFB03B05DF804FB00BFAC030120F2
:10D4EC00202302491A46024805F0B4BAC816012096
:10D4FC00CC030120002337B5094D01930120FFF720
:10D50C007FFE0446FFF7E2FD00220023284601A916
:10D51C0003F078FB08B1002CF0D1019803B030BDBA
:10D52C00CC030120002307B50022019306480023F9
:10D53C0001A903F067FB10B1FFF7DCFF0190019824
:10D54C0003B05DF804FB00BFCC030120F0B5037AF7
:10D55C00457A85B00190D8074FEA15151CD4DDB17A
:10D56C00002426463146019804F07EFD0746FFF75D
:10D57C0039FE70B134B9019B2946186904F091FC4D
:10D58C00044648B124FA06F3D90702D53846FFF70A
:10D59C0091FF0136AE42E5D3019B1A7A920704D56E
:10D5AC005B69084C0393039B2BB9064801A903F054
:10D5BC005BFB05B0F0BD1D68204603A903F054FBCE
:10D5CC000395F0E7CC0301200EB403B503AB53F87D
:10D5DC00042B014604480193FFF724F902B05DF8CF
:10D5EC0004EB03B0704700BF792401002DE9F04F24
:10D5FC0011F0020485B0904606461A469DF8387024
:10D60C0001F0010901F0080507D011F0440F37D1E2
:10D61C003249FFF7D9FF01460C46B9F1000F0AD089
:10D62C002F4B304653F827202E4B2F49002A08BF8A
:10D63C001A46FFF7C9FF3DB12C4B304653F8272053
:10D64C002B49FFF7C1FF0546B8F1000F43D001236A
:10D65C0003FA07F7274B17F0100F274F18BF1F4679
:10D66C00BDF840109DF83C00FFF73CFD39460246E2
:10D67C003046FFF7A9FF2844204405B0BDE8F08FE1
:10D68C001E4B19680029C7D01D4B4FF4616E1B68E7
:10D69C004FF47A7CB2FBF3F3B3FBF1F4B4FBFEF280
:10D6AC000EFB124E01FB14340CFB04F4B4FBF1FB27
:10D6BC004FF03C0A01FB1B440CFB04F4BEFBFAF3D9
:10D6CC00B4FBF1F1CDE901B10AFB13E100910D4975
:10D6DC00FFF77AFF9FE7084FC2E700BFB83301009E
:10D6EC00B8300100AA3301001E390100CC30010012
:10D6FC00DD330100B4330100AF330100E803012036
:10D70C00EC030120C133010038B50C46E107054696
:10D71C0003D5084A0849FFF757FFE20608D4A306C9
:10D72C002846BDE838404CBF04490549FFF74CBFBB
:10D73C0038BD00BFAA3301001E39010009330100B6
:10D74C00083301002DE9F0471D46089B1746DA0601
:10D75C0004460E4605D499064CBF2A492A49FFF7C0
:10D76C0033FF4FF00008DFF8A890A8452ADB00250E
:10D77C00DFF8A080DFF8A090DFF894A0BD422FD294
:10D78C0049462046725DFFF71FFF0135102D20D151
:10D79C0020461E49FFF718FF0025DFF87480DFF8DC
:10D7AC007C90AF4228D9725D4946A2F120035F2BD1
:10D7BC0028BF2E222046FFF707FF0135102D14D16C
:10D7CC00BDE8F08749462046FFF7FEFE08F1010848
:10D7DC00CBE76A07D2D151462046FFF7F5FECDE7DD
:10D7EC0041462046FFF7F0FECFE76B07D9D1414603
:10D7FC002046FFF7E9FED4E741462046FFF7E4FE5A
:10D80C00DBE700BF0933010008330100ED330100F1
:10D81C00EB330100E9330100E3330100EF33010086
:10D82C002DE9F0478B7A174613F0070805460E468C
:10D83C000A7A8AB021D0D2434989C3F3C203C1F317
:10D84C008911CDE900830291F368394602F0010297
:10D85C00FFF7CCFE8146347AE44314F001040ED079
:10D86C002946304604F098FCB8F1000F2BD0424604
:10D87C0039462846FFF748FF25E0C146EBE7B8F1EB
:10D88C00000F26D12746EB6806AA069330463B4686
:10D89C00A96804F06DFC069A6B681A603AB1AB6823
:10D8AC00134413F8014CA4F10A035C425C41284672
:10D8BC0004F0CFFD069B1F44002BE4D11CB128467D
:10D8CC001349FFF781FE284604F0C3FD0AB0BDE8FA
:10D8DC00F087304604F0F6FB0E4902462846FFF767
:10D8EC0073FE4FF0100A05AA2346304606A9CDF860
:10D8FC0014A004F03DFC059A002AB8D04B462846EB
:10D90C00009706A9FFF71EFF059B1C44EBE700BF21
:10D91C00F23301001E39010042F20F7373B58B42D2
:10D92C0028BF0B4605680446052168460D4A04F0DD
:10D93C0093F80646636828460B225B680A4904F094
:10D94C001EFC63683246694628465B6804F017FC87
:10D95C0063681B2228465B68044904F010FC02B083
:10D96C0070BD00BF873C010030340100143401004D
:10D97C0001230021074A10B5074C1360A04204D8BC
:10D98C0001B11360054B186010BD012140085B000C
:10D99C00F4E700BFEC03012040420F00E803012034
:10D9AC00F8B50D460446064F4618B44201D1284638
:10D9BC00F8BD386814F8011B83685B689847F4E776
:10D9CC0004040120014804F044BD00BFF8300100FC
:10D9DC000148FFF7A1BF00BFF830010008B50348AC
:10D9EC0002F08EFF024B186008BD00BF3C340100F2
:10D9FC000404012010B50C46084604F029FB21460E
:10DA0C0004480F22FFF70CFF2046BDE8104004F03D
:10DA1C004ABB00BFF830010010B5074802F070FF98
:10DA2C00064C074B1860204601F040F82046FEF7E4
:10DA3C00EBFD002010BD00BF3C34010051DA0000AA
:10DA4C00080401200A2838B50446074D04D128687B
:10DA5C0083680D215B68984728688368E1B25B682E
:10DA6C009847204638BD00BF0804012070B5044615
:10DA7C000C250D480E46231A9A100C4B402153438B
:10DA8C00DBB25D4305F14003184404F00FFD011EA9
:10DA9C0004DB074B2B445B68984700212046334638
:10DAAC00BDE87040184700BF1C040120B76DDBB601
:10DABC001C3101002DE9F0410F4C104D031B9B1044
:10DACC005D43EBB20C255D43074605F140000E4665
:10DADC002044402104F003FD011E08DB084B2C44BC
:10DAEC00C4E90E36074B5B59BDE8F0411847384680
:10DAFC003346BDE8F04118471C040120B76DDBB676
:10DB0C004D2501001C31010070B500220121044695
:10DB1C00052000F0B5FA052000F094FA0F4802F049
:10DB2C00A1F80F4B984215D104F01EFFE6680D4981
:10DB3C00304603F0EDFF00280BDB01253564E4686B
:10DB4C00084904F11C0003F0E3FF002801DB00206E
:10DB5C00E56470BD6FF00400FBE700BFA9DB0000BB
:10DB6C000000AD0B3431010001460C2300224B4365
:10DB7C00084870B5C4184033D4E90E561844A26353
:10DB8C0004F0CBFC2DB132462B46BDE87040024868
:10DB9C00184770BD1C0401201001012010B1012890
:10DBAC0004D07047034B1B6C5B0701D1FFF7DCBF44
:10DBBC00704700BF1C04012008B54FF02003EFF3A1
:10DBCC00118183F31188BFF36F8F114A136843F0EF
:10DBDC00020013F0010310600BD00E4AD2F80C3483
:10DBEC00D2F80C2413F0010303D00B4804F095FC7D
:10DBFC00012381F31188BFF36F8F23B1BDE8084077
:10DC0C000020FFF7B1BF0120BDE8084002F03AB890
:10DC1C006C040120005000405C040120074BD3E849
:10DC2C00EF2F22F00201C3E8E01F0028F7D1D30741
:10DC3C0002D4012002F058B8704700BF6C040120D8
:10DC4C001FB500220123CDE902236B46084ACDF80B
:10DC5C0000D0CDF804D004F099FC002805DB4FF47B
:10DC6C0080420023684603F0A3FB05B05DF804FB7B
:10DC7C006B2501002DE9F843012207463649D1E80E
:10DC8C00EF3FC1E8E02F0028F9D133B933493448CC
:10DC9C004B60CB608A6003F04EFF7B1E012B2ED8AD
:10DCAC00012F06D12F4BD3F81C3403F00303022BA6
:10DCBC0025D004F0B6FF044618B92B4B1B78002B6B
:10DCCC0044D14FF02003EFF3118683F31188BFF397
:10DCDC006F8F0124234DDFF89C80A946D5F81834AA
:10DCEC00D5F81824D2030CD503F00303022B01D072
:10DCFC00012F06D134B386F31188BFF36F8FBDE8C3
:10DD0C00F883D4B1304600F01BFAD5F81835DBB2E5
:10DD1C00012BE3D1D8F80020002ADFD00022C8F86C
:10DD2C000020D8F8002002222021C5F818250F4A1F
:10DD3C00C2F880110E4A1360D0E70021212003F0B5
:10DD4C00EFFAE2E70223C9F80433D8E70222054BC5
:10DD5C000646C3F80823BDE7700401200C0401201B
:10DD6C003804012000500040E105012000E100E0F2
:10DD7C000850004004510040044A1368C81A20F0AF
:10DD8C007F400344136003F00FBD00BF80040120EB
:10DD9C002DE9F0474FF480374FF00009860000F171
:10DDAC00500406F18046A40006F5A836A4B204F18E
:10DDBC008044D6F84035DFF86C8021F07F4504F5BF
:10DDCC00A8348740D8F804A5A3EB0A0323F07F43BB
:10DDDC002AF07F42012BC6F8402502D1132004F013
:10DDEC0026FF0AF10202AB1A23F07F43B3F5000FB2
:10DDFC0088BF1546C4F80090236825F07F43C8F807
:10DE0C004473C6F84035D8F804359A4506D0EB1A59
:10DE1C00023B23F07F43B3F5000F01D8BDE8F08738
:10DE2C002B46CFE700500140F8B5002427460F4E93
:10DE3C000F4B104A18461D6804B1F8BDD2F80413F4
:10DE4C00C903FAD531680029F7D0346031684FF432
:10DE5C008031C2F848130124D2F8401525B10020B6
:10DE6C005A681F60A847E3E70560E6E740510140A8
:10DE7C00740401200050014038B500244FF4803365
:10DE8C004FF400120D4D0121C5F80845C5F80433B7
:10DE9C000B4B1520C3F88021224600F0F1F8152019
:10DEAC0000F0D0F80123074A02201360064A2B60C9
:10DEBC001360FFF7DFFE204638BD00BF0050014065
:10DECC0000E100E0085001407C040120134BB0F14C
:10DEDC00FF3F08BF1846013800281CDD9842A8BF38
:10DEEC0018460F4BD3F804250E4B1968521A12F42E
:10DEFC00000F18BF002022F07F4301330A4A03446D
:10DF0C000A48106000205060044A934294BFC9181C
:10DF1C008918FFF73DBF0020E3E700BFFFFF7F003C
:10DF2C0000500140800401207404012085DD0000B4
:10DF3C004FF02002EFF3118382F31188BFF36F8F40
:10DF4C00064AD2F80405064A1268801A20F07F406F
:10DF5C0083F31188BFF36F8F704700BF00500140EF
:10DF6C00800401204FF02003EFF3118283F311881A
:10DF7C00BFF36F8F0649074B0868D3F8043582F35B
:10DF8C001188BFF36F8F1B1A23F07F43184470471F
:10DF9C008004012000500140094A0A49936809682D
:10DFAC009867D96708494B6843F080534B6000234E
:10DFBC0083F31188BFF36F8F9368D86F704700BFDE
:10DFCC0098050120D432010000ED00E013498A6865
:10DFDC004FF038001044EFF3098C80E8F01F20203C
:10DFEC0080F31188BFF36F8F0D4F4FF000668A6A74
:10DFFC008A603E60906F0023936780F3118802F172
:10E00C00380090E8F01F8CF3098802F1000004B589
:10E01C0004F0DCFABDE804407047000098050120CC
:10E02C0004ED00E01EF0040F0CBFEFF30880EFF3DB
:10E03C000980816911F8021C0229FFD001B504F096
:10E04C00C9FA01BD43B2002B08DB012200F01F000E
:10E05C0002FA00F0024A5B0942F82300704700BF45
:10E06C0000E100E0054B420953F82220012300F0A7
:10E07C001F0003FA00F01040704700BF00E100E001
:10E08C0043B2002B01F10101ACBF03F16043064B1D
:10E09C004FEA4111C9B2ABBF03F5614300F00F0069
:10E0AC0083F800131954704714ED00E042F8203C3B
:10E0BC00009B0B4942F81C3C019B21F0010142F8EA
:10E0CC00183C029B42F8081C42F8143C4FF0807339
:10E0DC0042F8043C0023203A82658367704700BFF6
:10E0EC00D51B0100044608B50E46154600F03EFB54
:10E0FC00084B9C60A36E83F30B88284686F3098833
:10E10C00002163B681F31188BFF36F8F00220023C7
:10E11C0003F05AFD98050120014910220A6070474E
:10E12C0010ED00E072B6404080F31188BFF36F8FA2
:10E13C00BFF34F8F30BF62B6BFF36F8F704700BF16
:10E14C0072B6494081F3118820BF80F3118862B602
:10E15C00704700BF73B506460C4601B3134B144D04
:10E16C001448ED1AED08AD0145F00105ADF800506D
:10E17C00D1E90123096803F0EEFEADF80050D4E9B3
:10E18C000423E1680C4803F0E6FE2A46E1690B48DB
:10E19C0003F0B4FE2A46A169094803F0AFFE2146FC
:10E1AC00304602B0BDE8704002F0D2BBEC2F01004B
:10E1BC002C30010084340100B3340100E23401003E
:10E1CC00F134010030BFFFF7FDBF00BF0E4A08B5A8
:10E1DC000E4B22F07F029A60BFF34F8FBFF36F8F0D
:10E1EC00D3F8882022F47002C3F88820EFF314834C
:10E1FC0023F0040383F3148802F03CFC03F0DCF9F5
:10E20C0000F086FA02F05AFC00C0000000ED00E0BD
:10E21C0001B572B60B4A506A00281EBF002151622C
:10E22C0004F016FC62B6EFF30580A0F110004FEA83
:10E23C00C0000549014409C99847BDE8014003499C
:10E24C000847000098050120E42D0100DDE60000E0
:10E25C0003F002FE202080F3118808484FF400617F
:10E26C00401880F30988EFF314800221084380F3EF
:10E27C001488BFF36F8FFFF7A9FF0000280E012051
:10E28C00EFF30880EFF3098101B5724600F040F915
:10E29C0001BD00BF70B5284B284C294DE41AE40889
:10E2AC00A40144F001063146264803F01AFEAA6A7E
:10E2BC00930103D53146244803F013FEAB6ADD010C
:10E2CC0004D5224844F0010103F00BFE1C4DAE6A4C
:10E2DC0016F4801605D01E4844F0010103F001FE2F
:10E2EC000226AB6A180304D51A4844F0010103F066
:10E2FC00F8FD134DAA6A510304D5174844F00101E7
:10E30C0003F0EFFDAB6A9A0304D5144844F0010105
:10E31C0003F0E7FD0A4DAB6ADB0304D5104844F06B
:10E32C00010103F0DEFDAB6A30466FEA03436FEA8E
:10E33C001343AB6270BD00BFEC2F01002C30010009
:10E34C0000ED00E01F350100373501004A350100B2
:10E35C00643501008E350100AC350100D13501006A
:10E36C00EB3501002DE9F041284B294C294DE41ADD
:10E37C00E408A40144F0010807460E46264841462D
:10E38C0003F0AFFDAA6AD00603D54146234803F03B
:10E39C00A8FDAB6A190704D5214844F0010103F02C
:10E3AC00A0FD1C4DAB6A9A0712D544F001084146FA
:10E3BC001C4803F096FD696BAB6A1B0608D54246F8
:10E3CC00194803F09BFD1FB1AB6A23F08003AB62CD
:10E3DC00104DAA6AD00704D5144844F0010103F08B
:10E3EC0080FDAB6A990604D5114844F0010103F095
:10E3FC0078FD0020074B9A6AD20658BF9A6A9A6A2F
:10E40C0042F0FF029A623070BDE8F081EC2F0100FF
:10E41C002C30010000ED00E0163601002C36010016
:10E42C005F360100723601008A360100A036010009
:10E43C00BF3601002DE9F0412A4B2B4C2B4DE41A31
:10E44C00E408A40144F0010807460E46284841465A
:10E45C0003F047FDAA6AD10403D54146254803F0D1
:10E46C0040FDAB6A1A0504D5234844F0010103F0C2
:10E47C0038FD1E4DAB6A9B0512D544F00108414690
:10E48C001E4803F02EFDA96BAB6A180408D5424652
:10E49C001B4803F033FD1FB1AB6A23F40043AB629E
:10E4AC00124DAB6A590504D5164844F0010103F02E
:10E4BC0018FDAB6ADA050DD5134844F0010103F0E1
:10E4CC0010FD0020094A936A43F47F439362307035
:10E4DC00BDE8F081AB6A9B04F3D50C4844F0010114
:10E4EC00EDE700BFEC2F01002C30010000ED00E047
:10E4FC00EE360100043701005F36010015370100CC
:10E50C002E370100433701005E370100BF36010092
:10E51C002DE9F0435A4B0746D3F80480894614463C
:10E52C0000258BB0C8F3080685F31188BFF36F8FF5
:10E53C0002F07F43B3F17F4F23D1D00721D4510692
:10E54C0003D422070ED401250EE04E494E4B4F4802
:10E55C005B1ADB089B0143F0010103F0C2FC14F0D1
:10E56C00040501D04F46002500238DF80730F31E1B
:10E57C00092B6CD8DFE803F0075A5E3E6B6B6B6BB4
:10E58C006B622F46F0E74FF000083E4B3E4E404882
:10E59C00F61AF608B60146F00106314603F0A1FC66
:10E5AC00374B8DF80780DC6A14F0020405D0314635
:10E5BC00384803F096FC00241FE0DB6A5B001CD596
:10E5CC003146354803F08DFC344B1B782BB10120C0
:10E5DC000DF10701FFF7C6FE0EE0314B1B782BB196
:10E5EC0001200DF10701FFF725FF05E02D4B1B88DE
:10E5FC009BB213B1FFF74EFE04469DF8073093B95A
:10E60C002022394602A804F051F8099B9DB3C3F3AC
:10E61C00080222B96FEA53236FEA43230993204679
:10E62C0002A9FFF797FD0BB0BDE8F08300200DF1B8
:10E63C000701CFE700200DF10701D4E71249114B78
:10E64C001948C91AC908890141F00101B1E70D4AFD
:10E65C000D4B16489B1ADB0818F4F87F4FEA83130E
:10E66C00134943F0010318BF0146A6F110021148EB
:10E67C0003F058FC9FE723F4FF7323F00103CDE76D
:10E68C0000ED00E0EC2F01002C300100763701008A
:10E69C0099370100B0370100D137010028ED00E0B7
:10E6AC0029ED00E02AED00E0F03701003B380100D5
:10E6BC002638010054380100044B5A6942F010020C
:10E6CC005A615A6942F480625A61704700ED00E069
:10E6DC00044B9968986A884203D003494FF08052E2
:10E6EC000A6070479805012004ED00E0BFF34F8FDE
:10E6FC000549064BCA6802F4E0621343CB60BFF3D2
:10E70C004F8F00BFFDE700BF00ED00E00400FA05ED
:10E71C00002320210348C2180133412B82F8001337
:10E72C00F9D1704700E100E008B50E4B9B688342BD
:10E73C0007D1EFF3058393B10B4A536843F0805331
:10E74C00536002F083FC4FF02003EFF3118083F34E
:10E75C001188BFF36F8FBDE8084004F0B6B902F022
:10E76C000BFF00BF9805012000ED00E01FB5094C20
:10E77C00094A23460121094800F038F90023039384
:10E78C00074B0121E41A01A80193029400F038F917
:10E79C0004B010BD00000420000001204031010035
:10E7AC00D801012010B50B680C7A23F01F0204F07D
:10E7BC001F031A43CB68640923F01F03044943EA7F
:10E7CC00440343F001038860CA600B6110BD00BFB5
:10E7DC0090ED00E00F2810B50DD9084B084A014602
:10E7EC00D21AD2089201074842F0010203F086FBCC
:10E7FC006FF0150010BDFFF7D5FFFBE7EC2F010004
:10E80C00243001006B3801002DE9F04F8946144685
:10E81C0006464FF00008544D85B0C84533DAD6F89B
:10E82C0004A0BAF1000F4DD0BAF11F0F1ED91AF087
:10E83C001F0F1BD1D6F800B01BF01F0F16D1584676
:10E84C0003F0ECFE07460AEB0B00013803F0E6FE82
:10E85C0087421CD06FF01507444A454B3946D21AF3
:10E86C00D2089201434842F0010208E041463F4A77
:10E87C003F4B4148D21AD208920142F0010203F0F8
:10E88C003DFB6FF01504204605B0BDE8F08F17F185
:10E89C00160FE1D0631EBB42DEDBAF60E968AF60F0
:10E8AC002B6921F01F0143F01F0BD6E900321A44EB
:10E8BC00994202F1FF3A1AD1D34507D13146F8B249
:10E8CC0003F093FE08F101080C36A6E73146AF6061
:10E8DC00EB6822F01F0203F01F031A43EA60E0B258
:10E8EC0003F083FE10F1160FCBD0441CEAE7013B7A
:10E8FC00D345E0B223F01F03AF6006D12A6931463D
:10E90C0002F01F0213432B61EAE7296901F01F0192
:10E91C000B432B61314603F068FE10F1160FB0D09B
:10E92C00AF60EA689DF808300BF1FF3B62F304031B
:10E93C008DF808302B699DF808205B0863F34712AB
:10E94C008DF80820D6E900321344009323F01F03FE
:10E95C005B44A3EB0A03013023F01F036946C0B2EA
:10E96C000393FFF737FFBDE790ED00E02430010083
:10E97C00EC2F0100B4380100913801000522034B43
:10E98C005A60BFF34F8FBFF36F8F704790ED00E06D
:10E99C00BFF35F8F0022014B5A60704790ED00E08F
:10E9AC0038B50E4C2568102D14D8FFF7F1FF002058
:10E9BC000B4B0C4A1A63854205D10B4B1D70FFF7AC
:10E9CC00DDFF002038BD616801EB0011FFF7EAFEA6
:10E9DC000130F0E74FF0FF30F4E700BF4C3101009D
:10E9EC0090ED00E0AAFF4400DF05012010B5034CB8
:10E9FC002278FFF709FF207010BD00BFDF05012052
:10EA0C002DE9F74F264D8A4606464FF00008AB46D7
:10EA1C00244FD0451BDAD6F80490B9F1000F39D049
:10EA2C0031680846019103F0F9FD0199044609EBA0
:10EA3C000100013803F0F2FD84424FF014021A4B2E
:10EA4C0008D06FF0150302FB08F84BF8083003B040
:10EA5C00BDE8F08F14F1160F2C60F8D01978A14294
:10EA6C00F5DD02FB08B0BC60BC60FC6800F108017D
:10EA7C00007B64F30400087138690C79400860F37A
:10EA8C0047140C71F96821F01F016960396921F094
:10EA9C001F01296108F1010814350C36B9E700BFD4
:10EAAC008404012090ED00E0DF050120014B18608B
:10EABC00704700BF0800012000F01F02054800EB62
:10EACC008200D0F8003223F4403343EA0143C0F80B
:10EADC00003270470025844008B5094B1A786AB992
:10EAEC000121312019700521FFF7CAFA3120FFF7F7
:10EAFC00A9FA4FF00042034BC3F80423002008BDD1
:10EB0C00E0050120001003402DE9F3410E46416859
:10EB1C0006F01F07097AB2F5A03FD0F80C8047EA3F
:10EB2C0041170AD1624807F01F01803150F82110BB
:10EB3C00C90708D56FF022009DE0B2F5005FD8F848
:10EB4C000C1000F09B800121D8F80C00B14001435F
:10EB5C00C8F80C100121D8F81400B140B2F5A03F50
:10EB6C000CBF08438843C8F814000020D8F81820BC
:10EB7C00B3F5C02F0CBF0A438A43C8F81820D8F845
:10EB8C001020B3F5802F4B4D0CBF114322EA01012D
:10EB9C00C8F81010D5F80433DBB200F5A27255F8A2
:10EBAC002220C2F3042297426DD123FA00F2D2073D
:10EBBC0069D5830003F1804303F54433D3F8102562
:10EBCC0022F00102C3F8102501238340C5F8083355
:10EBDC00C0B201F01BF938460021FFF76DFFD8F8E1
:10EBEC000C00F04010F0010045D0D8F81400F040B3
:10EBFC0010F001044ED0D8F818300DF10700F34096
:10EC0C00DB0757BFD8F81010032621FA06F606F0DA
:10EC1C0001065CBFC6F10206F6B201F019F9264BEB
:10EC2C00984234D19DF807103F028B0003F18043CA
:10EC3C0003F54433D3F8102507F4F85722F4473280
:10EC4C0022F44072C3F81025D3F81025880017431E
:10EC5C001A4A47EA064602440020C3F810651060C1
:10EC6C001268D3F8102542F00102C3F810250123D5
:10EC7C008B40C5F8043302B0BDE8F0810120B040F0
:10EC8C0021EA000164E70130082886D1A3E76FF080
:10EC9C001200F0E7D8F810103846F14001F00101ED
:10ECAC00C1F10301C9B2FFF707FF2046E3E700BF3C
:10ECBC0000258440001003400000AD0B0011034000
:10ECCC00284B70B546682848134083423BD00DD87A
:10ECDC00062B15D005D89BB1022B36D06FF0150042
:10ECEC0030E0B3F5801FF9D1012309E01F488342BE
:10ECFC002DD0B3F5A00F2CD0B3F5800FEED102239D
:10ED0C00D0064CBF0325C2F3401582F4807412F474
:10ED1C00007FC2F34020C4F3002406D012F4006F2D
:10ED2C00766818D001228A40B26040EA4402002082
:10ED3C0042EA032301F01F010D4A43EA85038031A7
:10ED4C0042F8213070BD0723DAE70423D8E7052306
:10ED5C00D6E70323D4E7520542BF01228A40F26072
:10ED6C00E3E700BF0600F0000600100002004000C0
:10ED7C00002584402DE9F8433F4F3E68002E4FD0CC
:10ED8C004FF001084FF000093C4BDD68D3E9052139
:10ED9C000A4325EA02053A4A1B6914695C4025EAD4
:10EDAC00040475BB3D603B68002301251F463548B4
:10EDBC003549D0F8042305FA03FC1CEA020F0FD0E6
:10EDCC0051F8232062B103F5A27250F8222041F8C9
:10EDDC002370C2F3042205FA02F2144351F82320E3
:10EDEC000133082BE5D1ECB94EB101260027234D98
:10EDFC00EC68D5E905210A4324EA020454BBBDE8BA
:10EE0C00F88315EA080F06D0002109F01F00FFF760
:10EE1C0053FE25EA080509F101094FEA4808C0E745
:10EE2C003446C1E7154B59680029DDD00D68174FE2
:10EE3C00002D38BF00258A68224002D038464B6826
:10EE4C009847002DD0D02B682946002B38BF0023C3
:10EE5C001D46F0E726420CD0296907F01F00F94047
:10EE6C0001F00101C1F10301C9B2FFF725FE24EA4B
:10EE7C00060401377600C1E77C1103409804012099
:10EE8C000025844000100340001103405001012074
:10EE9C0010B50446002201210A20FFF7F1F8606842
:10EEAC00E3680C4A00F1080101F042FA0A4B98425F
:10EEBC000DD00A4B0A4A0B48D21AD208920121688B
:10EECC0042F0010203F01AF86FF00F0010BD0020A1
:10EEDC00FCE700BF49EF00000000AD0BEC2F010078
:10EEEC000C30010001390100CA0708B543680FD482
:10EEFC00C1F34202012A0ED0022A15D00C490D4B47
:10EF0C000D48C91AC908890141F0010102F0E9FF55
:10EF1C006FF0150007E04FF0CC721B68C3F8242586
:10EF2C00C3680020596208BD4FF0C8621B68F5E742
:10EF3C000C300100EC2F0100213901000378012B6A
:10EF4C0008D0022B08D04BB9054B0B6201F1100015
:10EF5C0002F00EBA034BF8E7034BF6E7034BF4E76A
:10EF6C000000AD0B0100AE0B0200AE0B0100AD0BAF
:10EF7C002DE9F04F934614221D46C4688BB006460B
:10EF8C0089460DEB02000021D4F82C80B4F828A09F
:10EF9C0003F0B7FB8DF815504FF0FF324FF0FF33F5
:10EFAC00204602F005FAF0681030002700220023FA
:10EFBC0002F0FEF9706801F001FA4D463C465F45DF
:10EFCC0001D3002449E0297A0B0700F1A580BAF19E
:10EFDC00000F0DD07B1C9B450AD9880708D42B7DCC
:10EFEC0081EA030202F0010203F0040313431FD071
:10EFFC00002C3CD100242B6808936B6806932B7A69
:10F00C00706803F0010213F0020F8DF8142005A9AB
:10F01C000CBF2022002201F0FDF9414B98423AD05E
:10F02C000B3398420CBF6FF00F046FF0040414E024
:10F03C0001236A68101950451BD93A493A4B3B4891
:10F04C005B1ADB089B0143F001032146ADF800304D
:10F05C00534602F080FF6FF01B04706801F0BEF99C
:10F06C00F06802F085F920460BB0BDE8F08F002364
:10F07C00DFE7C90706D4296808EB0400039303F003
:10F08C0015FB039B6A68144483BB002CB2D0CDF8EB
:10F09C0020800694B3E7F06810304FF480420023D0
:10F0AC0002F086F968B1204A1E4B3946D21AD208B2
:10F0BC0092011F4842F0010202F020FF6FF004049D
:10F0CC00CBE7F368196A164B99420BD0154A164BCD
:10F0DC0018489B1ADB089B013A4643F0010302F0E7
:10F0EC0021FFEBE72B7ADB0703D4002401370C3527
:10F0FC0065E7089B9845F8D10C2303FB07935A68E6
:10F10C000C3B9442F1D3A41AD86808EB0401039386
:10F11C0003F0CCFA039BF2E76FF022049DE700BFEB
:10F12C000000AD0BEC2F01000C3001003339010055
:10F13C00553901007F39010000210248C2E9000164
:10F14C00002070470024F400002310B504464068EA
:10F15C001A4600F1080100F0B3FE094B98420DD09D
:10F16C00084B094A0948D21AD2089201216842F088
:10F17C00010202F0C3FE6FF00F0010BD0020FCE78F
:10F18C000000AD0BEC2F01003C30010001390100F7
:10F19C002DE9F04F89B09DF848600F46144699460A
:10F1AC00D0F80480C568002E40F0998008F1070261
:10F1BC0012F8013FFF2B04D023F080039F4200F094
:10F1CC0091800136F6B2042EF2D1684A684B39466A
:10F1DC00D21AD2089201674842F001025AE000228A
:10F1EC00009294E00132042A40F09F8021460022D4
:10F1FC00B1F5004FD0B23FD2A873D8F800002C6004
:10F20C00A981C0F80C25C0F804C5C0F808154C45F8
:10F21C00A34628BFCB46AA7B03F400432BFA02F18A
:10F22C000B43AAF804305249504B07925B1ADB0887
:10F23C0051499B01CDE9031743F0040305224F48C4
:10F24C0003A9CDE905B402F0A2FEBAF80430C3F369
:10F25C000E0313B1AA899A421FD808EB060393F93F
:10F26C00082007F01F07464BBBF1000F19D04C4587
:10F27C0077D8002A17DB74E00132082A4FEA5101D3
:10F28C00B6D12146394A3A4B3E48D21AD20892019D
:10F29C0042F0010202F032FE5CE0009B93B90020C8
:10F2AC005AE04C455BD8012101FA07F7DF6029468B
:10F2BC00304603F099FA0028F1D10146404603F09C
:10F2CC0081FBECE7404600F0BBFE0028FAD002239D
:10F2DC000122404608F1180100F074FEDFE76FF0E0
:10F2EC00220039E005EB460ABAF80430C3F30E02EB
:10F2FC001AB1A98991423FF672AF29463046019363
:10F30C0003F072FA80F00100C3B20093019B98F8ED
:10F31C000EC02A68BCF1010F04BF64084FEA5909FA
:10F32C00A2423FF474AF0022281DD1B2B1423FF487
:10F33C0059AF30F81210C1F30E0100293FF452AF4F
:10F34C000A490B4B1048C91AC908890141F001013F
:10F35C0002F0C7FD6FF0150009B0BDE8F08F002A70
:10F36C00A1DA012101FA07F79F60A0E73C30010008
:10F37C00EC2F0100233A0100703A0100F33901002F
:10F38C0000258440C9390100B439010038B5044660
:10F39C00002201210B20FEF773FEE3680E4ADC64A9
:10F3AC00606800F10C0100F05FFE0C4B984211D02C
:10F3BC000B4B0C4A2168D21AD20892010A4842F02F
:10F3CC00010202F09BFD6FF00F05E06803F056FAA6
:10F3DC00284638BD0025F8E721F700000000AD0BEA
:10F3EC00EC2F01004C30010001390100F0B5C5686B
:10F3FC0085B02B6CAC6C7BB99CB9002228461146AD
:10F40C0003F017FAAC6205F1180001F0B1FF00230C
:10F41C0085F8543005B0F0BD002C35D09C4228BF87
:10F42C001C46E96B466879B173B101F06043B3F1E6
:10F43C00005F09D0082C28BF082405F15507224687
:10F44C00384603F033F93946B268EB6B944228BF67
:10F45C00144600912C651BB12B6C002B18BF234656
:10F46C0001936B6C02931BB1AB6C002B18BF234642
:10F47C00002269463046039300F09CFE034B9842F1
:10F48C00C8D06FF00404B8E71C46CAE70000AD0B07
:10F49C002DE9F74F1E468B8880465B040D461746B8
:10F4AC00C4682DD44FF0FF324FF0FF3304F1080045
:10F4BC0001F07EFF6560D8F80C2013689D4200F0C7
:10F4CC00B280AB88D80722D5834A844BD8F8001079
:10F4DC00D21AD2089201824842F0010202F00EFDCB
:10F4EC006FF0150523689B8813F4804304D1636087
:10F4FC0004F1080001F03CFF284603B0BDE8F08F92
:10F50C002369002BCED163689942CBD1D3E719077D
:10F51C000AD57149714B7348C91AC908890141F060
:10F52C00010102F0DEFCDBE713F4C05F08D06A498E
:10F53C006A4B6D48C91AC908890141F00101F0E70D
:10F54C00C3F34513082B08D06349644B6748C91AA9
:10F55C00C908890141F00101E3E72968644B99422C
:10F56C0008D85D495D4B6348C91AC908890141F047
:10F57C000101D6E7AB68D8F804901560002B7CD05D
:10F58C001868002879D093F809A0197A1AF0010F9D
:10F59C000CBF4AF4B05A8AF4206AD0F80CB08368D5
:10F5AC0052461B680191984768B901230199DBF811
:10F5BC00002003FA01F11AF0010F14BF114322EAE3
:10F5CC000101CBF80010A988D9F80020880701F0B8
:10F5DC0004035DD5002B14BF03230223022BC1F3BC
:10F5EC00001159D0032B5AD0012B01D141F002014B
:10F5FC00414BC2F854152968994253D93F4B994253
:10F60C0053D93F4B994253D93E4B994253D93E4B18
:10F61C00994253D93D4B994234BF4FF080414FF042
:10F62C000041C2F82415012384F85430002F48D02F
:10F63C003B687A68E36222631A685B68E26323645E
:10F64C00002E43D0336872686363A2631A685B68E8
:10F65C006264A364002201212046A26203F0E9F84F
:10F66C004046FFF7C3FE4FF0FF324FF0FF3304F17B
:10F67C00180001F09DFEA56A34E7184B1649244882
:10F68C00C91AC908890141F0030102F02AFC9AE762
:10F69C00003B18BF0123A1E741F00401A8E741F0AA
:10F6AC000601A5E74FF00071BBE74FF08061B8E7AA
:10F6BC004FF00061B5E74FF08051B2E74FF00051C9
:10F6CC00AFE7C4E90B77C4E90F77B9E7C4E90D6676
:10F6DC00C4E91166BEE700BF4C300100EC2F0100FD
:10F6EC00813A0100A33A0100C23A0100E53A010057
:10F6FC0047E80100143B01008FD003001FA1070055
:10F70C003F420F007F841E00FF083D0000127A006C
:10F71C00453B010010B503780C46002B4ED10B6C09
:10F72C0063B10A6D9A421DD92549264B2648C91A40
:10F73C00C908890141F0010102F0D3FBA36C63B14C
:10F74C00226D9A4224D91E491E4B1F48C91AC9085A
:10F75C00890141F0010102F0C4FBE06CBDE81040EE
:10F76C00FFF744BE9B1A0B6463B90B6B013B0B6335
:10F77C0063B1CB6A03F10802CA629A68DB68CA6398
:10F78C000B64DBE7CB6B002BD8D01344E363D5E7DA
:10F79C009B1AA36463B9A36B013BA36363B1636B53
:10F7AC0003F1080262639A68DB686264A364D4E7BD
:10F7BC00636C002BD1D013446364CEE710BD00BF43
:10F7CC004C300100EC2F01006B3B0100F0B54B7984
:10F7DC00012B29D0032B24D110268B79032B20D17C
:10F7EC00CC7924B1012C1CD143681B79CBB10A799B
:10F7FC0012B1022A15D10E220B684568B3F5164FCB
:10F80C002D6865D02DD8B3F5165F64D016D8B3F536
:10F81C00966F62D00AD8B3F5967F61D0B3F5167F98
:10F82C0061D06FF0220052E00026D6E7B3F5166FD8
:10F83C005CD0B3F5965FF4D1374B3CE0B3F5E14FB8
:10F84C0057D007D8B3F5615F55D0B3F5964FE8D1D3
:10F85C00324B30E047F61227BB42E2D14FF40003A3
:10F86C0029E0B3F5613F48D013D8B3F5963F47D0A4
:10F87C0009D84DF6C027BB4244D0B3F5614FD0D167
:10F88C004FF46B0317E0B3F5E13FCAD14FF0EB73C4
:10F89C0011E0B3F5612F38D008D8214FBB4237D0D7
:10F8AC00B3F5E12FBDD14FF0E86304E01D4FBB422F
:10F8BC00B7D14FF08053C5F82435C3683443224385
:10F8CC00043303C9C5F86C2583E803000020F0BDA0
:10F8DC004FF41D03EFE7144BEDE74FF49E23EAE7DB
:10F8EC004FF4A033E7E74FF41C33E4E74FF41D2348
:10F8FC00E1E70E4BDFE70E4BDDE74FF06C73DAE719
:10F90C000C4BD8E74FF46503D5E74FF07063D2E7A3
:10F91C004FF08063CFE700BF00B0130000A04E0093
:10F92C0090D0030040420F000050270000C075002B
:10F93C0000F03A0000903A012DE9F0410646884665
:10F94C00C76803F06EF9B8B9284B1B7883F0010334
:10F95C007268156893B14FF02003EFF3118483F3B1
:10F96C001188BFF36F8F304602F0D9FF38BB84F398
:10F97C001188BFF36F8FEEE70123E9E7642430466B
:10F98C0002F0CDFF70B9012002F0ECFF013CF6D182
:10F99C000021212001F0C4FCF0E784F31188BFF3AF
:10F9AC006F8FF5E74FF02003EFF3118483F3118889
:10F9BC00BFF36F8F304602F0B2FF0028EDD0012369
:10F9CC00002207F8108FC5F84475C5F84835C5F8FE
:10F9DC002021D5F82011C5F85821D5F85821AB6055
:10F9EC0084F31188BFF36F8FBDE8F081E10501202E
:10F9FC004FF0000C43682DE9F041C6681C680F46B7
:10FA0C00C4F800C50546306008680121414B00F080
:10FA1C001F02914099600321803243F822107A68CA
:10FA2C00511C1EBF02F01F01803143F821C0B96880
:10FA3C00C4F80C05481C18BF0020C4F814251EBFC0
:10FA4C0001F01F02803243F82200F868421C0CD0EF
:10FA5C004FF0010C00F01F020CFA02FCC3F808C0B6
:10FA6C004FF0030C803243F822C0C4F80805C4F8E8
:10FA7C001015E96828460431FFF7A8FE8046A8B99E
:10FA8C006B689B7913B306F1120000F0A1F9224BBD
:10FA9C0098420ED0214B22492248C91AC908890123
:10FAAC0041F0010102F01DFA6FF004084046BDE878
:10FABC00F081B37C43F00043C4F8A031C4F88C301F
:10FACC000123B27C9340184AC2F804350823C4F8C9
:10FADC0000357B6801330CD00023C4F81031D4F806
:10FAEC00103106F11103C4F834350123C4F838354C
:10FAFC0023606B689B791BB94FF48073C4F8043393
:10FB0C0000231036C4F84465C4F848350123A360BB
:10FB1C00E360CBE7002584400000AD0BEC2F010027
:10FB2C00543001009D3B01000070014030B585B0A0
:10FB3C006C460546084B0FCB84E80F0000220121D0
:10FB4C000820FEF79DFA0820FEF77CFA214628468D
:10FB5C00FFF74EFF05B030BD7030010030B585B0F9
:10FB6C006C460546084B0FCB84E80F0000220121A0
:10FB7C000920FEF785FA0920FEF764FA214628468B
:10FB8C00FFF736FF05B030BD8030010008B5FDF73A
:10FB9C006DFC064B06490748C91AC908890141F092
:10FBAC00010102F09EF90020FEF7A0FDEC2F0100F0
:10FBBC00FC2F0100D33B01002DE9F0430025214C23
:10FBCC00214E54F8048CDFF8889085B0A84503D8F2
:10FBDC00002005B0BDE8F083636A96E807001F6853
:10FBEC0001AB83E807000C221946384602F04EFDA3
:10FBFC0090B98FB1636A21691B681A6991420BD164
:10FC0C009A69A169914207D8E169914204D9626964
:10FC1C005B6932EA03030AD0276A67B10B4801F02B
:10FC2C000EFF404080F311884FF0040002DFE368C0
:10FC3C0001351C44CAE7484601F001FF636A1F60A6
:10FC4C00F5E700BF3CC2000090300100F03B010022
:10FC5C00193C0100014B024A1A6070470401012053
:10FC6C000090D003044B1A7922B9012218601A7142
:10FC7C000248704702487047B40401200000AD0BE5
:10FC8C000C00AD0B10B101281ED07047134BD3F8EC
:10FC9C001824D3F8181411F4803F194610D002F030
:10FCAC000302022A0CD1C3F8182500220C4B1A604F
:10FCBC0002221B68094BC3F8042301229A60704787
:10FCCC000123C1F81835F0E70022064B1A601B68B7
:10FCDC00024BC3F804031860704700BF005000408B
:10FCEC00045100400051004038B510B1012816D025
:10FCFC0038BD0222012142F21075164CC4F80823BB
:10FD0C00154A10601268154A1160D4F81834DB03D8
:10FD1C00EED5012002F026FE013DF6D1E8E70022E7
:10FD2C0042F210750E4B0B4CC4F808031A601B689A
:10FD3C000C4B1860D4F80C34D4F80C2403F00103E9
:10FD4C00D203D5D5002BD3D0012002F00BFE013D00
:10FD5C00F0D1CDE700500040045100400C50004061
:10FD6C000051004004500040154B10B51A684AB1C0
:10FD7C000020012218601B68124BC3F80823124B99
:10FD8C001B689847114B1A6882B100221A601B68D5
:10FD9C000C4BD3F81824D3F8181402F00302012AE0
:10FDAC004FF0020103D1C3F818159A6010BDC3F8C7
:10FDBC000813054B0120BDE810401B68184700BF15
:10FDCC000051004000500040B40401200451004098
:10FDDC000B4A70B51668F14389B271B10025ECB2CB
:10FDEC0021FA04F3DB0705F10105F8D50123A34043
:10FDFC00334304700348136070BD0348FCE700BF35
:10FE0C00BC0401200000AD0B0200AD0B012303FA72
:10FE1C0000F010F0FF0F12D04FF02003EFF3118120
:10FE2C0083F31188BFF36F8F064AD36C23EA00006B
:10FE3C00D06481F31188BFF36F8F03487047034878
:10FE4C00704700BFC00401200000AD0B0400AD0BD7
:10FE5C002DE9F041FF22002401260546DFF858E089
:10FE6C001448DFF85880E3B24FF02001EFF3118C07
:10FE7C0081F31188BFF36F8F22FA03F1C9070AD5FA
:10FE8C00DEF84C1006FA03F7394201BF40463943FD
:10FE9C00CEF84C102B708CF31188BFF36F8F40454C
:10FEAC0005D006FA03F39A4304F10104DBD1BDE853
:10FEBC00F08100BF0200AD0BC00401200000AD0BAF
:10FECC002DE9F04F0C2605793A4C6E43A71997F89B
:10FEDC0008C085B0BCF1000F6AD17B604FF0010AFD
:10FEEC006B464FF0030BDFF8D8E0A25101F1FF3C59
:10FEFC0001F103091CF8017FFF2F55D027F0800674
:10FF0C001E600E7B6EB907F01F060AFA06F83F0654
:10FF1C0006F180064CBFCEF80880CEF80C804EF867
:10FF2C0026B0CC4503F10403E4D10068009BC0F873
:10FF3C006035019BC0F86435029BC0F86835039BA3
:10FF4C00C0F86C350123C0F800358E790B894F79D8
:10FF5C00C0F80C75C0F80465C0F808354B89C0F8BA
:10FF6C0010350023C0F80032C0F80033C0F81C3143
:10FF7C00D0F81C11C0F81031D0F81011C0F81431A1
:10FF8C00D0F81411C0F80431D0F804311AB140F390
:10FF9C000730FEF757F80C2303FB054401230648F2
:10FFAC00237205B0BDE8F08F4FF0FF361E60B8E746
:10FFBC000248F6E7100501200000AD0B0500AD0B63
:10FFCC0000258440F0B40D461C4601791B4B01EB17
:10FFDC0041010068D5F800C0AF88AE6803EB810121
:10FFEC00EB68C0F820C5C0F82475C0F82865C0F8C7
:04FFFC002C35C0F8E8
:020000021000EC
:1000000040C5C0F84475C0F84865C0F84C3502F0EA
:10001000010303EB5202C0F81425E20711D414F0D7
:10002000020203D0002B14BF08220422002BC0F8C8
:10003000002218BF0C23E2B208BF0823F0BC02F074
:10004000A4BC1022F2E700BF100501200C21084BD0
:10005000027901FB02320168137AD1F80411DBB294
:1000600019B9981E18BF01207047012010727047FF
:1000700010050120944624222DE9F04705794C4EC5
:100080006A43B418277F002F40F0908000686360B7
:100090000124012746F802C091F8008091F80CE095
:1000A000444B08F01F029440BEF1010F02F18002A0
:1000B00094BFDC609C6043F822704A78FF2A1FBF1F
:1000C00002F01F04A740DF6003271CBF803443F801
:1000D00024708F7808BF4FF0FF32FF2F1FBF91F8B9
:1000E0000E9007F01F044FEA8909803418BF43F8C7
:1000F00024904FF0240909FB0569CC7808BF4FF024
:10010000FF37FF2C89F81F4016D04FF0010A91F8F5
:10011000049004F01F040AFA04FAB9F1000F3CD06D
:10012000C3F80CA04FF0030A803443F824A0242322
:1001300003FB056383F81E908B68C0F80885C0F840
:100140000C25C0F81075C0F824354B7B003B18BF58
:100150000123BEF1020F23D0BEF1030F23D0BEF165
:10016000010F01D143F00203C0F854358B79C0F878
:10017000C0350723C0F80035BCF1000F03D040F3B1
:100180000730FDF765FF242303FB056500236B772C
:10019000012309482B77BDE8F087C3F808A0C1E721
:1001A00043F00403E0E743F00603DDE70348F2E72A
:1001B00040050120002584400000AD0B0500AD0B7B
:1001C00024232DE9F0410679434F73431446FA186E
:1001D0000D46517F864600297BD1FB5823B114F090
:1001E000140F04BF012353774FF0240C95E80F0040
:1001F0000CFB067C0CF10C0888E80F009CF81F3003
:10020000FF2B08D003F01F0201239CF81E1093401F
:10021000324AB1B19360296821B101F06043B3F172
:10022000005F06D1AA6872B102F06043B3F1005FCB
:1002300009D0242303FB0676002329487377BDE801
:10024000F081D360E7E7DEF800306868C3F8441552
:10025000E968C3F84805C3F834250022C3F8381507
:10026000C3F81821D3F8182114F0010218BF012295
:10027000C3F8502514F0020218BF012214F008013F
:10028000C3F8402504BF01221A6124227243BA58E0
:10029000B2B919B9D3F81821002AFBD0242303FBE3
:1002A0000676F37FFF2B07D003F01F020123B17FF7
:1002B00093400A4A11B1D3600A48C0E79360FBE754
:1002C000402214F0040F14BFC3F80823C3F804231A
:1002D000F2E70548B3E700BF400501200025844050
:1002E0000A00AD0B0000AD0B0B00AD0B0F4BD3F8AC
:1002F0001821CAB10022C3F81821D3F818310C4BC9
:10030000DA7FFF2A07D002F01F010122987F8A407E
:10031000084938B1CA60002207485A771A72D3E9EF
:10032000002110478A60F6E7704700BF00B0004028
:100330004005012000258440480501204FF0340C81
:10034000F8B506791C4D0CFB06FC05EB0C0494F883
:100350002D707FBB40F20C6EA760636084F82F7035
:100360004B7B84F830700F6884F8323045F80C20ED
:1003700007F01F03DFF84CC080334CF823E04C68D3
:10038000006804F01F0380334CF823E08B68C0F84A
:100390000875C0F80C45C0F824351AB140F3073091
:1003A000FDF756FE342303FB06550123034885F869
:1003B0002D30F8BD0248FCE7640501200000AD0BBC
:1003C0000500AD0B00258440062102680379C2F8C0
:1003D00000153421034A01FB0323022283F82D2058
:1003E000704700BF640501200268037934200A4980
:1003F00000FB0313002009499860C2F80813D2F8E3
:10040000001221F4BC51C2F80012C2F8000501220A
:1004100083F82D20704700BF6405012002029C0173
:100420002DE9F0473426002390F804E0AE4F04682D
:1004300006FB0E7686F82E30CB680D4603F060433F
:10044000B3F1005F944603D0A84E3046BDE8F08774
:10045000A74BC4F8083396F82F3003F0FF0A23B1F6
:10046000B368A44EC4F80433EFE712F0140F0CBFC6
:1004700001230023894686F82F3006F10C08B9E8DD
:100480000F00A8E80F00D9F80030C6F820C0C8F85F
:100490000030CCF3001386F830306B78C4F8883520
:1004A000C4F804A1D4F80431C4F824A1D4F8243148
:1004B000C4F860A1D4F86031C4F848A1D4F8483138
:1004C0001CF0010318BF0123C4F850351CF00203CF
:1004D00018BF0123C4F840352B78032B00F2B280FB
:1004E000DFE803F0819D66022A6902F06043B3F100
:1004F000005FA9D14FF48073E968C4F800326B68DB
:10050000C4F84415C4F848350023C4F85031D4F871
:10051000501101212162A160D4F850110029FBD0B3
:10052000C4F85031D4F85031AB68C4F84425C4F84D
:10053000483534234FF4802203FB0E739A6008235E
:100540006D4E1CF0080F04D12A78032A1CBF01222B
:10055000E250342303FB0EF3FA18FB58002B74D13E
:100560000125D4F84821D4F80411002940F08780EF
:10057000003A18BF0122D4F82411002900F0858028
:10058000C4F82431D4F82411D4F86001D4F800124E
:1005900010B111F4007F04D1256265610028E0D01C
:1005A0000022C90571D5C4F84831D4F84821D8E7EC
:1005B0006B68EA68C4F84425C4F848352B6903F031
:1005C0006042B2F1005F7FF43FAFAA68C4F83435EF
:1005D0004FF48453C4F83825C4F80032342302227F
:1005E00003FB0E7312E06B68EA681CF0200FC4F87E
:1005F0004425C4F848354FF034030BD04FF48072D3
:10060000C4F800224FF4802203FB0E739A6001238A
:10061000236294E74FF40072C4F80022DFE76B68AE
:10062000EA68C4F83425C4F838354FF48053C4F868
:1006300000323423022203FB0E739A6001232362EB
:1006400000237DE708232D4E7BE71CF0040F1CBF21
:10065000002393601CF0400F06D1342303FB0E737C
:100660009A6842F002029A60342303FB0E77BB685B
:1006700043F40073BB60BB68C4F80433E5E6C4F818
:100680000431D4F80421012275E7002A3FF469AF50
:100690003421002001FB0E72D4F8C434C4F8C434F1
:1006A00082F82F008BB1164A13F0010F154E18BFB8
:1006B000164613F0020F02F1010218BF164613F09E
:1006C000040F114B18BF1E46BFE61CF0400F7FF40D
:1006D000BCAE20460EFB017102F090F9094B0028D8
:1006E00008BF1E46B1E600BF640501200A00AD0B3D
:1006F00002029C010B00AD0B0000AD0B0400AD0B22
:100700000000AE0B0100AD0B0200AE0BF0B55B4B71
:100710005B4CD3F824211D4687B0FAB10022C3F800
:100720002421D3F82421D3F80421BAB9A268C3F84C
:1007300008230222A260A268C3F80423D3F8602130
:100740001AB1D3F800329E0503D401224B4B1A6232
:100750005A61012384F82E3007B0F0BDD5F804317A
:10076000002B54D00023C5F80431D5F80431236A96
:100770005D060AD494F82E303BB941493F4802F057
:100780003DF980F0010084F82E00236A13F004077D
:1007900022D13C4E01AD0FCE0FC5336894F830C066
:1007A0002B60364BC3F86071D3F86021C3F85C71DD
:1007B000D3F85C21BCF1000F02D094F82E205AB17E
:1007C0000022C3F80022A2602F4AC3F808234FF486
:1007D00080622E4BC3F88021284AD2F8C43498078F
:1007E000C2F8C4343CD501238DF8003094F8303081
:1007F0000BB984F82F30236A5B0703D594F82E30A9
:10080000002BA9D0D4E9003168469847A4E7C5F881
:100810004831D5F84831237B83B91A4F01AE0FCF49
:100820000FC63B68336094F83030002BD4D1C5F844
:100830000032A360144BC5F80833C8E74FF40073C7
:10084000C5F8003240F20223A36003F1CE73C5F86D
:100850000833A368C5F804330123AB602B627BE740
:10086000590701D50223BFE7DA0701D50323BBE708
:1008700094F82E30002BB7D00423B5E700A0004039
:10088000640501207005012002029C0100E100E0E6
:10089000F8B5104B104F53F82050013053F820603A
:1008A000AE4200D8F8BDD5E900342046984770B173
:1008B0006CB10123E41B094A2411610952F821009B
:1008C00004F01F0403FA04F4044342F821400835FD
:1008D000E6E700BFC032010010010120C001012085
:1008E000084BC01A0011084B420953F8222001237B
:1008F00000F01F0003FA00F010420CBF1846002061
:10090000704700BF10010120C0010120114970B5DE
:1009100005460E46104C8C4204D10F4CB4420AD10D
:10092000002414E02046FFF7DBFF10B12368AB4240
:100930000DD01034EFE72046FFF7D2FF08B910348E
:10094000ECE72846216801F09BFE0028F7D12046FD
:1009500070BD00BFC0010120100101202DE9F3414D
:1009600006460F464FF02003EFF3118883F31188FA
:10097000BFF36F8F00F0FCFC214C224B042EA4EB44
:1009800003044FEAD40498BF1F4A4FEA841444F08A
:100990000103054694BF52F826201C4AADF80030EA
:1009A000314600231A4801F0DCFA47B1FB69C3F372
:1009B000080323B1174844F0010101F098FA44F00C
:1009C00001042DB1284602F03FF908B1037803B9BC
:1009D0001148FCF7DBFB2346024629460F4801F08D
:1009E000A7FA39463046FFF7D7F888F31188BFF3E6
:1009F0006F8F284602B0BDE8F041FDF79BBE00BFF7
:100A00002C300100EC2F0100D83201004C3C0100D9
:100A1000623C01008A3C01005A3C0100AB3C0100F1
:100A2000F8B505460027154E4FF02002EFF311836D
:100A300082F31188BFF36F8F286988B12F6183F328
:100A40001188BFF36F8F00F007FB4FF02003EFF327
:100A5000118083F31188BFF36F8F02F03CF8E3E756
:100A600002F00AF9012104460228D8BF084602F024
:100A700013F97462FDF75CFBD6E700BF980501200F
:100A80000248034A0021121A01F041BED801012098
:100A9000E4050120012208B5094B02201A70FFF776
:100AA000F7FE00F083FD0320FFF7F2FE00F00CFDDF
:100AB000FBF742FD034A137B23F00103137308BDC8
:100AC000E1050120100301202DE98048A7B0FCF7C3
:100AD000C1FA344B03F5006989F3088883F30A8867
:100AE0000024E023304D4FF0010B85F82230EC77E5
:100AF0002C766C76AC766B6A2C4E43F4E0236B62FA
:100B0000FDF7E0FDFDF70EFB4FF0FF33AB62EB624C
:100B100040F20113264DADF8243006ABAB60204601
:100B2000CDE92044FFF7B4FE0120FFF7B1FEDFF866
:100B300098A000F0A1FB1F4BAE624FF480621E49EB
:100B4000059330465346CDE9034BCDE9014400946B
:100B500000F05EFC737B804623F004033046737321
:100B600001F0E5FF0F23154F4FF4A072CDE90243CA
:100B70001349144B3846CDE904B4CDE9005400F0D4
:100B800047FC7B7B524623F004037B7305F11C0377
:100B900041463046C5E90733EF602C76C5F804902E
:100BA000FDF7A6FA280E012000ED00E01003012059
:100BB000980501200D3D0100E80801209002012068
:100BC000E80C0120210A0100950A010070B50E4BC6
:100BD0000E4CA34201D3002070BDD3E9030141EACA
:100BE000000212F003020BD19D685A61AA4201D1A2
:100BF0001C33EEE75E6901320E6059610144F5E78E
:100C00006FF01500E8E700BFC4010120C401012016
:100C1000D3B50C4616461F464FF02003EFF3118163
:100C200083F31188BFF36F8F43695BB123601B6847
:100C30004361836901338361002081F31188BFF32D
:100C40006F8F11E056EA070203D16FF00B002360AB
:100C5000F3E70246CDE90067044800F0BFFA18B98F
:100C6000034B9B685B69236002B0D0BDE2050120A5
:100C700098050120F8B504460D464FF02003EFF328
:100C8000118683F31188BFF36F8F47696FB901F045
:100C9000A9FF50B12A68C767426101F048FF314699
:100CA000BDE8F840074800F051B82B6862691A6047
:100CB0002B686361A369013BA36186F31188BFF3CD
:100CC0006F8FF8BDE205012010B5084C23685BB1B9
:100CD000FDF734F903462068054A03440021BDE8C6
:100CE0001040536101F0D8BF10BD00BFD4050120F2
:100CF00098050120F8B505460C464FF02003EFF3A8
:100D0000118683F31188BFF36F8F00224FF40047E1
:100D100040F2E73000210A4BE7FB05015A614FF42E
:100D20007A720023FBF78AFA064B1860064B1C60A8
:100D3000FFF7CAFF86F31188BFF36F8FF8BD00BFBE
:100D400098050120D4050120D005012049B9EFF311
:100D5000058030B9054B9A6A9B689A4201D0FDF72D
:100D600021B981F31188BFF36F8F70479805012077
:100D70004FF02003EFF3118183F31188BFF36F8FDE
:100D8000044B9A68D37B013BD37381F31188BFF383
:100D90006F8F704798050120094B03F12C028242A6
:100DA00005D19B688B4202D14B7BDB0606D1D1E992
:100DB000003213605A600023C1E90033704700BF5E
:100DC0009805012038B5124C01462369A2680BB181
:100DD000E5680CE004F12C0001F09FFE0546537B12
:100DE000980644BF43F008035373002DF0D049B96F
:100DF000537BDB0606D1AB6923B9D3897F2B01D99D
:100E0000A26238BD954201D0FFF75EFFA562F8E708
:100E10009805012010B54FF02003EFF3118483F300
:100E20001188BFF36F8F084B00209A68D37B013382
:100E3000D373FFF7C7FF84F31188BFF36F8FBDE84B
:100E4000104001F054BE00BF9805012070B490F925
:100E50000D20437B002A2CDBDB062AD1836943BBB0
:100E6000154A114651F82C4F8C4218BF2346002BCF
:100E700038BF0023146BB3B190F90E6093F90E5094
:100E8000AE4203DBA3420ED01B68F4E75A68C0E908
:100E9000003210605860437B63F07F03437370BC83
:100EA0000020FFF78FBFC0E90014136B18601063B8
:100EB000F1E770BC704700BF9805012010B54FF0F6
:100EC0002002EFF3118482F31188BFF36F8F427B0E
:100ED000510704D484F31188BFF36F8F10BD22F043
:100EE00004024273FFF7B2FF2146BDE810400148FB
:100EF000FFF72CBFE205012070B590F90D300146D7
:100F0000002B02DA1748FFF747FF174A104650F840
:100F10002C3F146B834208BF0023002B38BF0023F3
:100F2000D3B191F90E6093F90E50AE4203DBA342A8
:100F300012D01B68F4E75868C1E9003001605960BD
:100F40004B7B906863F07F034B73431A58425841C0
:100F5000BDE87040FFF736BFC1E90004136B1960AC
:100F60001163EDE7C405012098050120014670B525
:100F70004FF02003EFF3118483F31188BFF36F8FD9
:100F8000164B174A98681568A8421D4606D1FFF708
:100F90009BFE84F31188BFF36F8F70BD002616602F
:100FA000104A1268BAB1C2897F2A14D8427BD2068D
:100FB00011D10D4A90F90E60126896420BDB0B4A74
:100FC000904208D05A698A4202DCFFF795FFDEE7BB
:100FD000521A5A61DDE700236B61DAE798050120B8
:100FE000CC050120D4050120D0050120900201206C
:100FF00070B50446183001F029FE4FF02003EFF3DE
:10100000118683F31188BFF36F8F94F90D30002B95
:1010100007DA21460E48FFF7BFFE637B03F07F032C
:1010200063730C4D637BA86843F010036373031B69
:1010300058425841FFF7C6FE86F31188BFF36F8F01
:10104000AB68A34203D1BDE8704001F050BD70BD54
:10105000C4050120980501202DE9F04104464FF018
:101060002003EFF3118283F31188BFF36F8F437B6B
:1010700013F0280F05D082F31188BFF36F8FBDE8FE
:10108000F08143F02003437382F31188BFF36F8F25
:10109000183001F0DBFD4FF02003EFF3118683F3EE
:1010A0001188BFF36F8F637BD80616D1A269A2B9EE
:1010B000190607D521462648FFF76EFE637B03F02D
:1010C0007F036373234B9868021B50425041FFF724
:1010D00079FE002704F130081DE09B07F9D5214671
:1010E000A068FFF759FE637B23F0020363730023BC
:1010F000A360EEE705F1180001F0A8FDA8682946F5
:10110000FFF74AFE6B7B284623F002036B73AF6048
:10111000EF67FFF79BFE256B454501D0002DE9D118
:101120000C4B9A680C4B9A4202D10120FFF74AFE01
:10113000637B43F008036373236E86F31188BFF368
:101140006F8F002B9BD02046BDE8F041184700BFB1
:10115000C4050120980501209002012008B590F9EE
:101160000D300146002B06DA0748FFF715FE4B7BD2
:1011700003F07F034B73054B9868431A584258415C
:10118000BDE80840FFF71EBEC405012098050120F8
:101190002DE9F041064614461D464FF02003EFF3BB
:1011A000118783F31188BFF36F8F01F0F0FC87F391
:1011B0001188BFF36F8F6B1C08BFB4F1FF3F08D0DD
:1011C00022462B4606F118000349BDE8F04100F025
:1011D00063BABDE8F08100BF4F2B010010B50C468B
:1011E000064B11469868064B1860DDE90223FFF7AD
:1011F000CFFF2046BDE81040FCF7D4BE9805012083
:10120000CC0501202DE9F04105460F4601F05EFDB9
:1012100004464FF02003EFF3118883F31188BFF3E6
:101220006F8F124E124BB0682C441860FFF796FF78
:10123000B06810492A463B46183000F02DFAB268D3
:101240004046537B002543F010035373FCF7AAFE7E
:1012500001F03CFD241A65F10005002C75F1000336
:10126000B8BF00242046BDE8F08100BF98050120EA
:10127000CC0501204F2B01000021044B084603F14F
:101280002C02C3E90B22FFF735BD00BF98050120F2
:10129000F8B5244C244BA2689A4230D04FF020037A
:1012A000EFF3118583F31188BFF36F8FA16804F109
:1012B0002C00FFF771FDE36AA268834208BF002398
:1012C000002B38BF0023216B2BB392F90E7093F9DA
:1012D0000E60B74203DB8B421DD01B68F4E75968F0
:1012E000C2E900310A605A60537B012063F07F033A
:1012F0005373FFF767FD85F31188BFF36F8F4FF0CE
:101300002003EFF3118083F31188BFF36F8FBDE8E3
:10131000F840FCF747BEC2E90001236B1A60226364
:10132000E2E700BF9805012090020120B1F1FF3FE4
:1013300008BFB0F1FF3F08B502460B4606D10B4B84
:101340009868FFF755FE4FF0FF3008BD13430AD1F0
:10135000FFF79EFF00204FF47A7380FB0323D00B2E
:1013600040EA4340F1E7FFF74DFFF4E7980501201D
:10137000014B9868704700BF9805012038B50446B6
:101380004FF02003EFF3118583F31188BFF36F8FC4
:1013900001F028FC48B10022C26701F0C8FB2946D1
:1013A000BDE838400448FFF7D1BCD4E902329A4284
:1013B00018BF0133A360F2E7E205012037B51446F8
:1013C0001D464FF02003EFF3118183F31188BFF323
:1013D0006F8F836843B1013B836081F31188BFF352
:1013E0006F8F002003B030BD54EA050306D181F3AE
:1013F0001188BFF36F8F6FF00F00F3E70246CDE95E
:1014000000450248FFF7EAFEECE700BFE2050120D5
:101410002DE9FF4100F13005C0E90C550E9D044651
:101420000573042545730D9DD61D857300250C9A03
:1014300026F00706C0E90655C0E91A16C573056708
:1014400002920B9A01EB060801920A9A0092424618
:10145000FCF732FE054BC4E917559B6803B15B6F7F
:101460004046636704B0BDE8F08100BF98050120E5
:10147000F0B5002587B00595109DDDE9126704954C
:101480000F9D044603950E9D02950D9D01950C9DA3
:101490000095FFF7BDFF7B1C08BFB6F1FF3F05D0ED
:1014A00056EA070305D12046FFF708FD204607B09E
:1014B000F0BD32463B46034904F1180000F0ECF859
:1014C000F4E700BF4F2B01002DE9F0472A4E2B4DCA
:1014D000B04686B0B54205F1300410D3FFF748FCA2
:1014E0004FF4004940F2E7360027244CDFF890A083
:1014F000444521D306B0BDE8F047FFF78BBC54F854
:10150000043C059354F8103C049354F8143C0393A2
:1015100054F8183C029354F81C3C019354F8203CB6
:10152000009354E90A2354E90C01FFF771FF54F8C2
:10153000303CDD652546CDE7636A5A1C0DD0304648
:10154000394623EAE373C9FB0301B94208BFB0423D
:10155000256804D12846FFF7B1FC3034C8E74FF4C2
:101560007A720023FAF76AFE02460B4605F118006C
:10157000514600F091F8F0E7C4010120C4010120B8
:101580004F2B010008B54FF02003EFF3118483F3D4
:101590001188BFF36F8F044B98681861FFF728FD1F
:1015A0002046FCF7FFFC00BF98050120024A0349D2
:1015B000034800F04ABA00BF0A330100153D01009C
:1015C000223D010008B50648064A0749121A01F0F3
:1015D00073F8BDE80840054A0549064801F06CB8B3
:1015E00000000120D4010120503D01000000000056
:1015F000503D010000000120034B1B680BB9FCF7B4
:101600009DBC0020704700BFD805012030B503689D
:1016100068B10A4A5268904209D043B1D3E9042123
:10162000D0E90445121945EB0101C3E904214268E0
:1016300013605A600023C0E9003330BD0801012067
:1016400038B5134B1C689C4208BF0024FFF7D4FF39
:101650000546BCB1D4E90401401B61EBE5710128EA
:1016600071F1000311DB6FF000420023824273EB43
:10167000010400DA1046074B5B6913B19842A8BF1A
:10168000184638BD6FF00040F5E70020F3E700BFD3
:1016900008010120980501202DE9F74F0191194615
:1016A0004B1C08BFB2F1FF3F824670D06FF00103C0
:1016B0004FF0FF3B541C41F10005B3EB04086BEB0A
:1016C0000509B8F1000F79F100030FDBFFF794FF74
:1016D0006FF00103344AD2E9001C5B1A6BEB0C0279
:1016E0001E1B62EB0507341A67EBE075019BCAF815
:1016F00008304FF02003EFF3118683F31188BFF316
:101700006F8FFFF779FF012C75F10003BCBF012437
:101710000025264B24181A6845EBE0759A42CAE961
:10172000044501D05F6852B95A68CAF80030CAF857
:1017300004205A68C2F800A0C3F804A014E0D2E95B
:101740000489DAE90445444575EB090122DAB8EB6E
:10175000040069EB0501C2E904015168CAE90021EE
:10176000C1F800A0C2F804A01A689A420BD09245B2
:1017700009D1FFF765FF18B10D4B5B69834202D0B9
:101780000021FCF7A9FB86F31188BFF36F8F03B02C
:10179000BDE8F08FB4EB080065EB0901BA42CAE975
:1017A0000401C1D01268BEE79003012008010120A6
:1017B000980501202DE9F74F0646FFF7D7FB4FF0BC
:1017C0002003EFF3118483F31188BFF36F8FDFF8E9
:1017D000B0A02A4D5146DFF8ACB02E60D5F800C05D
:1017E000DBF800006246DAE90089D3175845CDE9F5
:1017F00000230DD060B1D0E90467B445BB411DDAC8
:10180000009BB6EB030C019B67EB0306C0E904C623
:101810000026009B2E6013EB0802019B43EB09039B
:10182000C1E90023FFF70CFF3146FCF755FB84F3B9
:101830001188BFF36F8F03B0BDE8F08F0022002343
:1018400018EB060849EBE679C0E90423ACEB060681
:10185000CAE900892E60FFF7D9FE84F31188BFF32F
:101860006F8F836898474FF02003EFF3118483F361
:101870001188BFF36F8F0249B0E700BFD805012080
:10188000900301200801012010B54FF02003EFF371
:10189000118483F31188BFF36F8FFCF74FFB064B66
:1018A000D3E90023121843F1000384F31188BFF336
:1018B0006F8F1046194610BD90030120F8B5D0E98E
:1018C0000A23561C43F10007002F08BF022E0446CE
:1018D00002D30C49FFF7E0FE236B01332363236A35
:1018E0000BB12046984754F8185FA54208D03DB187
:1018F000284601F0E0F8284601F019F90023EB67CB
:10190000F8BD00BFBD1801002DE9734F194606460A
:101910001046DDE90A234C1C08BFB0F1FF3F8046AA
:10192000894647D014461D4654EA050316D06FF089
:101930000103B3EB020A4FF0FF3363EB050BBAF17F
:10194000000F7BF1000309DA12F1FF3445F1FF3596
:10195000012C75F10003BCBF012400256FF00103C9
:101960001B1A00934FF0FF3363EB01030193DDE992
:101970000023002A73F100030CDA10F1FF3841F163
:10198000FF39B8F1000F79F10003BCBF4FF0000838
:101990004FF00009304601F059F900234246336305
:1019A00030464B460549C6E90A4502B0BDE8704FCE
:1019B000FFF772BE02B0BDE8708F00BFBD18010016
:1019C00038B5064C064DAC4201D3002038BD204648
:1019D000D4E9011201F0ACF91434F4E7C401012098
:1019E000C4010120034658B1426802F00302012AF3
:1019F00003D0032A04D1026812B100209860704716
:101A00006FF0150070474268034602F00302032A94
:101A10004FF00002816014BF104600685A607047A2
:101A20000020704730B58A680C68551C14B14B68AB
:101A3000934201DC8D6030BD013B934208BF002220
:101A40008D600CBFE254A054F5E70FB407B504A9AC
:101A500051F8040B0191FAF7E3FD03B05DF804EBD4
:101A600004B070470CB407B504AB53F8042B0193D2
:101A7000FAF7E4FD03B05DF804EB02B07047038BA6
:101A800013F0070305D10368002B0CBF00200320CF
:101A90007047022B05D1438B002B14BF002004207C
:101AA0007047012B05D10368002B0CBF00200520D7
:101AB0007047002070472DE9F0410D460746194652
:101AC000281D90461E46FFF79EFF044638B1334658
:101AD000424629463846A446BDE8F0416047BDE885
:101AE000F08110B44FF02004EFF3118284F31188D9
:101AF000BFF36F8F416110BC0121FAF7B3BD10B580
:101B00000C4640B139B1081DFFF76CFF28B9A36836
:101B100033F0030301D06FF0150010BD38B50C464B
:101B2000054658B151B10B6843B14B6833B11C2223
:101B3000002100F0ECFD00202C6138BD6FF0150095
:101B4000FBE770B504460E46FFF7D9FF051E31DBF3
:101B50004FF02003EFF3118183F31188BFF36F8FF0
:101B60004FF6FF75638B208BAB4200F007022ED03F
:101B7000022A0ED1013363831546012381F31188B4
:101B8000BFF36F8FB3B1002331462046FFF793FFB9
:101B900010E0830701D0062A0ED10023336063686A
:101BA00093B9C4E90066154662B90A462046022187
:101BB000FAF758FD284670BD052A0CBF6FF02205C4
:101BC0006FF004050023D9E71E606660EBE76FF055
:101BD0000A05F7E7044608B5084611461A46A04725
:101BE000FFF7C6FBFCF7A6FD836800EBC101B3F568
:101BF000004F2CBF51F8220031F81200704700EB63
:101C0000C1018068B0F5004F2CBF41F8223021F8A7
:101C100012307047012208B5FFF7E6FF400808BD03
:101C2000836800EBC101B3F5004F08D34B681AB1CC
:101C300043F001034B60704723F00103FAE74B8840
:101C40001AB143F001034B80704723F00103FAE718
:101C500053000122FFF7D3BF80680131B0F5004F78
:101C60002CBF02200120081AB0FA80F0C0F11F003A
:101C700070472DE9F04104460D46FFF7CBFFA368FE
:101C80000146B3F5004F01D3012835D02046FFF7B8
:101C9000E3FF04EB800216699EB9012303FA00F00A
:101CA000E36829460343E360204615612B46022280
:101CB000FFF7A5FF032229462046BDE8F041FFF7C4
:101CC0009EBF022231462046FFF78EFF074603469D
:101CD000022229462046FFF792FF33460322294677
:101CE0002046FFF78CFF032239462B462046FFF79C
:101CF00086FF02223146DFE7BDE8F081B2F5802F92
:101D0000F8B52CBF082504250023551B0022CC1D47
:101D100024F007040460C4E9002300230D4425F0E7
:101D200007052D1BED0829462046A560E360FFF757
:101D300093FF8600411C18461B36F60804F110027A
:101D40008B4229DB324620460021FFF781FFAF1B83
:101D5000204601220021FFF763FF3A463146FFF794
:101D600077FF3346314620460022FFF748FF2946D9
:101D700020460022FFF76CFF3B4629462046002202
:101D8000FFF73DFF294620460122FFF749FF314674
:101D9000BDE8F840FFF76DBF42F8040B0133CFE711
:101DA0002DE9F74F9946D37814466F2BA3F14102E2
:101DB00006460F4601922DD028D8582B14BF0A256D
:101DC0001025AA464FF0000BDDF8308052465B46E6
:101DD00030463946FAF732FA092AD3B21FD83033DF
:101DE0005F45DBB208BF564508F8013D01D3C84541
:101DF00012D823789B0605D5082D16D1A37843F079
:101E00000803A370404603B0BDE8F08F03F0F7036A
:101E1000702BD3E70825D4E706460F46D6E7019A8C
:101E2000192A94BF37335733DAE7102DEAD1A37854
:101E300043F01003E5E72DE9F041074688461546D3
:101E40001E461446B442A4EB050002D33EB92378E3
:101E50002BB1414614F8010BB8470028F2DABDE86F
:101E6000F0817047FDF7FCBE0023C0E900337047E6
:101E7000036823B90160002341600B607047436829
:101E80001960F8E7006870470346006808B1026807
:101E90001A60704708B5FBF74BFB18B1012343608C
:101EA0000023038108BDFCF763B800207047F0B53C
:101EB0000546002001270346024615F8014B0CB1E8
:101EC0008B4200D3F0BD252C02D182F00102F4E751
:101ED000002AF2D044F02006613E192EEDD8732C72
:101EE00004BF07FA03F2104301330022E5E738B5D7
:101EF00005460C46FFF7CEFF28B121460561BDE837
:101F00003840FBF737BA38BD70B506460D46144663
:101F1000FFF7C0FF58B10121427A066161F3071251
:101F2000427221464561BDE87040FBF723BA70BD9F
:101F30002DE9F04180460F4616461D46FFF7AAFFE1
:101F400068B10222437A294662F307134372C0E95B
:101F50000576C0F81080BDE8F041FBF70BBABDE88C
:101F6000F0812DE9F84380460F4616461D46BDF820
:101F70002090FFF78FFF70B10322437A494662F346
:101F800007134372C0E90576C0F81080C561BDE84B
:101F9000F843FBF7EFB9BDE8F88310B51C4600F035
:101FA00099F820B12146BDE81040FBF7E3B910BD18
:101FB0002DE9F8431C4603890E461146C3F38D02F2
:101FC000A2429DF8207003D800230B60BDE8F8837F
:101FD0000B682344934284BF131B0B600C2AD1F877
:101FE00000902AD9072CD0F814802DD80822183058
:101FF0004A4528BF4A462044154617B3314600F0EB
:102000005BFBA9EB05092E44B9F1000FDED0B8F156
:10201000000FDBD0C4F11C054D4528BF4D46201DE7
:102020002A464044BFB1314600F046FB0024D8F8B0
:102030000080A9EB05092E44E6E74FF000081430B4
:10204000D6E701463046DAE7083C1B2CDCD9D8F845
:1020500000801C3CF9E701463046E5E70430D0E853
:10206000EF3F0133C0E8E23F002AF8D17047407AE1
:1020700000097047437AB1EB131F4FEA131216D2CF
:10208000032A03D800EB810148697047012903D86E
:1020900000EB81018869704743690239062903D83A
:1020A00003EB8101486870471B680739F6E7002099
:1020B00070470346021DD2E8EF1F0139C2E8EC1F4A
:1020C000BCF1000FF7D15B680BB9FBF745BA70475D
:1020D000006970472DE9F84F814688461546FBF7A1
:1020E00027FA044630B301230027032D43600781FC
:1020F00009D90222A5F1020A028100F1140B4761FD
:10210000BAF1000F0EDC637A032D65F30713C4F8F0
:102110001090637218D84146AA0004F1140000F030
:10212000CBFA07E0FBF704FA064630B92046FBF786
:1021300013FA34462046BDE8F88FCBF80000AAF128
:10214000070A83460760DBE74146082204F11800CE
:10215000676900F0B1FA023D08F10808072D2E4624
:1021600028BF07264FEA86094146381D4A4600F037
:10217000A3FAAD1B3F68C844F0D1DBE713B50024D8
:102180000094FFF715FF02B010BDF8B506460D46E6
:1021900014461F46214628463A46B047241A0544AD
:1021A000F8D1F8BD2DE9F0478EB00EAF80460D4650
:1021B000FFF78EFF06464046FFF759FF4FF0000934
:1021C00082468300073323F00703ADEB030D0EAC0B
:1021D000D14516D14046FFF74AFF0F281ED8DFE849
:1021E00010F01900200026002D00360041004E009E
:1021F0005D006E0081009600AD00C600E100FE00AB
:102200001D0149464046FFF735FF44F8290009F112
:102210000109DDE731462846FBF7DCF9BD46BDE89C
:10222000F087314628462268FBF7D4F9F6E73146B5
:10223000D4E900232846FBF7CDF9EFE7A368314640
:1022400000932846D4E90023FBF7C4F9E6E7E368E6
:1022500031460193A36828460093D4E90023FBF795
:10226000B9F9DBE7236931460293E3682846019315
:10227000A3680093D4E90023FBF7ACF9CEE76369C8
:1022800031460393236928460293E3680193A368C8
:102290000093D4E90023FBF79DF9BFE7A36931461A
:1022A000049363692846039323690293E3680193C7
:1022B000A3680093D4E90023FBF78CF9AEE7E36948
:1022C00031460593A3692846049363690393236900
:1022D0000293E3680193A3680093D4E90023FBF71A
:1022E00079F99BE7236A31460693E369284605930B
:1022F000A36904936369039323690293E3680193D9
:10230000A3680093D4E90023FBF764F986E7636AC6
:1023100031460793236A28460693E3690593A36928
:1023200004936369039323690293E3680193A368A9
:102330000093D4E90023FBF74DF96FE7A36A314618
:102340000893636A28460793236A0693E369059313
:10235000A36904936369039323690293E368019378
:10236000A3680093D4E90023FBF734F956E7E36A46
:1023700031460993A36A28460893636A0793236A40
:102380000693E3690593A36904936369039323693F
:102390000293E3680193A3680093D4E90023FBF759
:1023A00019F93BE7236B31460A93E36A2846099300
:1023B000A36A0893636A0793236A0693E369059304
:1023C000A36904936369039323690293E368019308
:1023D000A3680093D4E90023FBF7FCF81EE7636BC6
:1023E00031460B93236B28460A93E36A0993A36A49
:1023F0000893636A0793236A0693E3690593A369C5
:1024000004936369039323690293E3680193A368C8
:102410000093D4E90023FBF7DDF8FFE6A36B314618
:102420000C93636B28460B93236B0A93E36A09931F
:10243000A36A0893636A0793236A0693E369059383
:10244000A36904936369039323690293E368019387
:10245000A3680093D4E90023FBF7BCF8DEE64268EA
:1024600010B5D2E90023044681680068FFF78DFEAD
:10247000002263681A6010BD38B54B6805461A68BB
:10248000CB680C469A4202D10846FFF7E8FF636822
:10249000D3E8EF2F511CC3E8E01F0028F8D1A36850
:1024A00000209D5438BDCBB20C21C26803FB012132
:1024B000086C00F0070070474FF02003EFF3118223
:1024C00083F31188BFF36F8F036813F0C00301D04B
:1024D0008B4207D101230360002082F31188BFF3F0
:1024E0006F8F70474FF0FF30F7E710B54FF02003C4
:1024F000EFF3118283F31188BFF36F8F036803F04A
:102500000704012C06D10160002082F31188BFF37B
:102510006F8F10BD03F0C0038B4214BF4FF0FF302C
:102520006FF04400F1E74FF02003EFF3118283F3E3
:102530001188BFF36F8F036803F0C00343F00203F9
:10254000036082F31188BFF36F8F704710B41C24AF
:10255000C068CBB203FB0400002110BC1047002070
:10256000FDF796BB0020FDF7C5BB1046FEF706BF82
:1025700038B50C24C9B24C430546C06804F1400389
:1025800080211844FFF798FF002804DB69680C4499
:1025900063689847002038BD2DE9F0410C24C9B28A
:1025A0004C43C568064604F140008021284490460B
:1025B0001F46FFF79AFF002806DB2544C5E90E8772
:1025C00073681B5998470020BDE8F0817047704739
:1025D00000210120FBF7C4BD836E83F30B88704795
:1025E00001460068FBF7BCBD08B5FBF7F1FDBDE88F
:1025F0000840FCF773B830B54B680C6885B00A89A1
:102600008D7A0094013B24F01F04234402F01F0242
:1026100042EA451223F01F0369468DF80820039310
:10262000FCF7DEF805B030BD40E800F313F4803F5E
:10263000D8B208BF6FF01500704770B50546013974
:102640002C4642B111F8013F561E2BB92A4404F81A
:10265000013BA242FBD170BD324605F8013BEFE7DA
:10266000034600201A5C02B970470130FAE70346BE
:1026700000201A5C0AB1884200D170470130F8E7A7
:10268000431E013913F8012F11F8010F824201D1C5
:10269000002AF7D1101A704710B55AB101398418C1
:1026A00010F8012B11F8013FA04201D09A42F7D057
:1026B000D01A10BD1046FCE7F0B581EA0004A5076A
:1026C00003460BD0013B0A4491421BD1F0BD002AC6
:1026D000FCD011F8014B013A03F8014B9C07F6D1ED
:1026E00022F003041D1F96080F19B94205D16FF09F
:1026F0000305234405FB0622E4E751F804CB45F823
:1027000004CFF2E711F8014B03F8014FDCE7034671
:1027100070B5C9B29C0711D141EA012422F0030629
:1027200044EA04451E449408B3420DD16FF00305FA
:1027300005FB04221A44934209D170BD002AFCD043
:1027400003F8011B013AE5E743F8045BECE703F803
:10275000011BF0E74FF0FF307047002070474368DF
:1027600000205B681B690B60704743685B685868B2
:1027700042400A4042405A600020704743680020AF
:102780005B6899607047436800205B68D960704758
:10279000436800205A6853684B4053607047C368D1
:1027A00030B5586858B10024814213D108685CB92B
:1027B0009C685860A14200D198600020086072B9FE
:1027C000002030BD2846EFE720609868814208BFAE
:1027D0009C60F2E705680446002DF3D13AB15A68CF
:1027E0000A60986859600028EAD19960E9E76FF0BB
:1027F0001500E6E7002330B50C1DDAB2824207D09F
:1028000034F81320C2F30E0212B18D89954204D818
:102810000133042BF1D1002030BD0120FCE701235E
:1028200003FA01F1C3681B68194218BF82F0010264
:1028300012B18368DB68184783681B69FBE738B50A
:1028400005680446FDB1AB68EBB11868D8B151B169
:10285000197A0122FFF7E3FF23689B685868BDE8F7
:10286000384000F0EAB912B9AA8892040BD458682B
:1028700000F0E3F9236800229B68197A1868BDE824
:102880003840FFF7CCBF38BD10B501220021044607
:10289000FFF7D5FF236933B9636004F10800BDE891
:1028A0001040FEF76BBD10BDC06810B503688B42C9
:1028B00006D190F8544034B9FFF7E6FF204610BD2A
:1028C0006FF01500FBE76FF00F00F8E743681B6837
:1028D000D3F80423D20518D5D3F82021AAB14FF09C
:1028E0002001EFF3118281F31188BFF36F8FD3F8CA
:1028F000201131B10021C3F82011D3F8201101219A
:10290000D96082F31188BFF36F8F70470B46C2689E
:10291000D2E9010183E803000020704743681B6887
:10292000D3F88004C3F88004704742681368D3F872
:10293000580138B9927932B9D3F82001003818BF5C
:1029400001207047012070474368C2681B68D3F8B4
:10295000100148B10020527C0A70C3F81001D3F86E
:10296000102101221A6070474FF0FF307047004776
:1029700000F063B908B50520FBF77AFB20B9BDE884
:1029800008400520FBF764BB08BD10B502244A725D
:102990000C72096871B112F0040F0CBF82219221F0
:1029A000140748BF41F02001D40648BF21F0800140
:1029B000C0F8001312064FF0000158BF0122C0F802
:1029C0000411D0F8044156BFC250C018084610BDCB
:1029D000002238B503680546C3F8002201225A6078
:1029E0000C46FDF733FB38B92846FDF72FFB18B925
:1029F000002CF9D1204638BD0124FBE70A7B0346B1
:102A0000032A29D8DFE802F0212519028A68500339
:102A100004D5D3F84C250869904207D18A6852033F
:102A20001AD4D3F84C254969914215D000200622CA
:102A3000C3F80005C3F800257047D3F84C25086992
:102A40009042F3D1D3F83C25EDE7D3F84C25096942
:102A5000EAE7D3F83C25FAE701207047FFF7B7BD56
:102A600030B50024846141EA020414F00304C0E993
:102A7000023201610CD14461A34203D1C0E90000DC
:102A8000002030BD456901340D6041611144F3E718
:102A90006FF01500F5E710B54FF02003EFF3118448
:102AA00083F31188BFF36F8F00F037F884F3118838
:102AB000BFF36F8F10BD10B54FF02003EFF31184FB
:102AC00083F31188BFF36F8F00F01BF884F3118834
:102AD000BFF36F8F10BD034620B9EFF305820AB92B
:102AE000FBF760BA83F31188BFF36F8F70474FF025
:102AF0002003EFF3118083F31188BFF36F8FFFF78B
:102B0000EABF014608B58068FEF746F94B7B23F023
:102B100002034B7300238B6008BD034600688342A9
:102B200003D0002838BF002070470020704710B540
:102B30004FF02003EFF3118483F31188BFF36F8FFD
:102B4000FEF784F984F31188BFF36F8F10BD70B561
:102B500004464FF02003EFF3118683F31188BFF38F
:102B60006F8F50F8103CA0F1180513B12846FFF7FD
:102B7000C8FF14F80B3C284623F0140304F80B3C60
:102B8000FEF764F986F31188BFF36F8F70BD38B517
:102B900004460D46FEF7E2FA637B43F002036373DB
:102BA000C5B12B68A5609D4208BF0023002B38BF2C
:102BB000002383B194F90E1093F90E20914204DBA7
:102BC0006A689A4207D01B68F3E75A68C4E9003282
:102BD00014605C6038BD6B68256063606B681C6066
:102BE0006C60F7E738B54FF02003EFF3118283F301
:102BF0001188BFF36F8FFFF790FF044682F31188AF
:102C0000BFF36F8F88B14FF02003EFF3118583F38B
:102C10001188BFF36F8FFFF774FF85F31188BFF33F
:102C20006F8F04F1180000F011F8204638BDEFF363
:102C30000580003818BF0120704708B1FAF7CCB9F9
:102C400070476FF0460070470020704710B54FF096
:102C50002002EFF3118482F31188BFF36F8F0368B2
:102C60003BB1FEF7D3FC002084F31188BFF36F8FD4
:102C700010BD6FF01500F7E710B54FF02003EFF32C
:102C8000118483F31188BFF36F8FFEF7D9FC84F3AF
:102C90001188BFF36F8F10BD70B504460D464FF01D
:102CA0002003EFF3118683F31188BFF36F8FFEF7D4
:102CB000C7FC012805DDA04203DD29462046FBF7BD
:102CC0000BF986F31188BFF36F8F70BD08B5FEF75F
:102CD000DBFD08BD0023C0E9081200F11802C0E9BD
:102CE0000622C0E9003303634363704710B504460E
:102CF000FFF7ACFFD8B9636A0BB12046984704F1DF
:102D000018000021FFF7C7FE044680B1FFF7D3FE8D
:102D10002046FFF70CFF4FF02003EFF3118083F301
:102D20001188BFF36F8FBDE81040FFF7D4BE10BD10
:102D300010B400F10C04C0E9034410BCFEF7DEBF80
:022D40007047DA
:022D4200FFFF91
:082D44002895FF7F010000004B
:102D4C00B1CF000000000000CD0B0100000000001E
:102D5C00C119010000000000ADE9000000000000F6
:102D6C0015DB00001001012069FB0000200101208F
:102D7C0039FB00003001012025DA000000000000C2
:102D8C0085DE000040010120EDCF000000000000B6
:102D9C00E5EA00005001012055F10000600101201E
:102DAC0055F100007001012055F100008001012057
:102DBC0055F10000900101209DEE0000A0010120C2
:102DCC0099F30000B0010120C5FB000000000000D9
:082DDC005B270100000000006C
:102DE40000000000D125010000000000D1250100F1
:102DF40000000000D125010000000000D1250100E1
:102E040000000000D125010075FD00006F290100BC
:102E140000000000D125010000000000D1250100C0
:102E240030010120CD28010020010120CD2801001E
:102E34000D0701006F290100ED0201006F29010057
:102E440000000000D125010000000000D125010090
:102E540000000000D125010000000000D125010080
:102E640000000000D125010000000000D125010070
:102E740000000000D125010000000000D125010060
:102E840000000000D12501000000000035DE000034
:102E940000000000D125010000000000D125010040
:102EA40000000000D125010000000000D125010030
:102EB40000000000D125010000000000D125010020
:102EC40000000000D125010000000000D125010010
:102ED40000000000D125010000000000D125010000
:102EE40000000000D125010000000000D1250100F0
:102EF40000000000D125010000000000D1250100E0
:102F040000000000D125010000000000D1250100CF
:102F140000000000D125010000000000D1250100BF
:102F240000000000D125010000000000D1250100AF
:102F340000000000D125010000000000D12501009F
:102F440000000000D125010000000000D12501008F
:102F540000000000D125010000000000D12501007F
:102F640000000000D12501000000000081ED0000F8
:102F740000000000D125010000000000D12501005F
:102F840000000000D125010000000000D12501004F
:102F940000000000D125010000000000D12501003F
:102FA40000000000D125010000000000D12501002F
:102FB40000000000D125010000000000D12501001F
:102FC40000000000D125010000000000D12501000F
:102FD40000000000D125010000000000D1250100FF
:082FE40000000000D1250100EE
:102FEC00E6380100030000006C340100030000000F
:102FFC00E43B010003000000FD3801000300000069
:10300C00A639010003000000A633010003000000F4
:10301C002C3301000400000067380100030000009D
:10302C00123D0100030000005434010003000000B5
:10303C00673A010004000000413301000300000066
:10304C008F3B010003000000C33B010001000000A6
:10305C00E0300100F00301204334010001000000C6
:04306C00FFFFFFFF64
:103070001200000013000000150000001400000002
:1030800016000000170000001900000018000000E2
:10309000DEE61E28EAAC45B8025B0000DEE61E282C
:1030A0004CBBCE8F025B000000000000000000005F
:1030B0000338FDD87047000000000000F433010021
:1030C000FC330100000000000000000000000000D0
:1030D00004340100083401000C34010010340100F4
:1030E00001DA00000000000000000000DDD900004F
:1030F000D1D90000E9D90000ADD90000F8030120C2
:10310000DE050120010000004DDC000071250100FA
:103110009925010000000000A7240100C5DB000084
:1031200029DC0000603401005F25010065250100F5
:1031300066340100C1DA000079DA00000000000006
:103140000000012000000000060001000200000055
:103150005431010000000000D738010006000000D3
:10316000E0FF0F0000000120DF3801002100000017
:10317000E0FF0320CDEC00005F2701006B2701007A
:103180007D270100872701009127010015EB000032
:103190009F27010000000000FFFFFFFF0025844083
:1031A00000000000F5EE00007DEF000000000000D0
:1031B000000000000000000000A00040000000002F
:1031C0000C0000000B0000000000400600000000A2
:1031D00000100240000000001D1E1FFF0004000040
:1031E000E80302010000000040000120040000008C
:1031F000000000000000000000200240010000006C
:103200001CFFFFFF00040000E803020100000000B3
:103210005000012004000000000000000000000039
:1032200000300240020000000D0E0F1000040000EC
:10323000E80302010000000060000120040000001B
:1032400000000000000000000040024003000000F9
:10325000FFFFFFFF00040000E80302010000000080
:1032600070000120040000000000000000000000C9
:103270009DF1000045F1000000B00040000000009A
:10328000FF0F0000030405FF0000FF0000000040E6
:10329000000000009DF40000A92801004929010058
:1032A00045F900001D290100D9F700000D29010092
:1032B0000080004006000100009000400600010070
:1032C0004C2D01008C2D0100942D0100DC2D0100FE
:1032D000E42D0100F5FFFFFFC33C0100D13C0100DC
:1032E000E53C0100F43C0100003D010050574D2039
:1032F0004170706C69636174696F6E2068617320DE
:1033000073746172746564210D0A0050574D5F300B
:10331000004469646E27742066696E64204C4544DD
:10332000206465766963652025730A006D6F647596
:103330006C65735F636F6D6D6F6E00286E696C29CD
:1033400000736F63006C6F6767696E67003C6C6F3A
:10335000675F73747264757020616C6C6F63206654
:1033600061696C65643E00617267756D656E74209D
:10337000256420696E20736F757263652025732044
:103380006C6F67206D6573736167652022257322FA
:10339000206D697373696E676C6F675F73747264B5
:1033A000757028292E006C6F67001B5B306D00253F
:1033B000733A200025732E005B2530386C755D2034
:1033C000005B253032643A253032643A253032646D
:1033D0002E253033642C253033645D20003C25736A
:1033E0003E2000253032782000202020007C00255F
:1033F00063000D001B5B313B33316D001B5B313BC8
:1034000033336D006572720077726E00696E66000C
:1034100064626700206D6573736167657320647211
:103420006F70706564202D2D2D0D0A1B5B306D00B3
:103430001B5B313B33316D2D2D2D200055415254F6
:103440005F30006C6F675F6261636B656E645F75B0
:1034500061727400706F77657200434C4F434B008C
:103460006866636C6B006C66636C6B00636C6F63A7
:103470006B5F636F6E74726F6C007379735F636CF4
:103480006F636B0072302F61313A20203078253025
:103490003878202072312F61323A20203078253060
:1034A0003878202072322F61333A2020307825304E
:1034B00038780072332F61343A2020307825303844
:1034C00078207231322F69703A20203078253038D8
:1034D00078207231342F6C723A20203078253038C1
:1034E000780020787073723A202030782530387850
:1034F000004661756C74696E6720696E73747275CD
:103500006374696F6E2061646472657373202872DE
:1035100031352F7063293A20307825303878002AE9
:103520002A2A2A2A205553414745204641554C54C2
:10353000202A2A2A2A2A0020204469766973696F82
:103540006E206279207A65726F002020556E616C62
:1035500069676E6564206D656D6F72792061636364
:10356000657373002020537461636B206F766572FE
:10357000666C6F772028636F6E7465787420617253
:103580006561206E6F742076616C6964290020206B
:103590004E6F20636F70726F636573736F72206913
:1035A0006E737472756374696F6E73002020496C5A
:1035B0006C6567616C206C6F6164206F6620455894
:1035C000435F52455455524E20696E746F205043EC
:1035D000002020496C6C6567616C20757365206FF5
:1035E0006620746865204550535200202041747451
:1035F000656D707420746F206578656375746520DF
:10360000756E646566696E656420696E7374727543
:103610006374696F6E002A2A2A2A2A204D50552089
:103620004641554C54202A2A2A2A2A002020537425
:1036300061636B696E67206572726F722028636FB9
:103640006E746578742061726561206D6967687455
:10365000206265206E6F742076616C696429002099
:1036600020556E737461636B696E67206572726F4B
:10367000720020204461746120416363657373208C
:1036800056696F6C6174696F6E0020204D4D464124
:103690005220416464726573733A20307825780053
:1036A0002020496E737472756374696F6E20416374
:1036B000636573732056696F6C6174696F6E002067
:1036C00020466C6F6174696E672D706F696E74202F
:1036D0006C617A79207374617465207072657365AA
:1036E00072766174696F6E206572726F72002A2A39
:1036F0002A2A2A20425553204641554C54202A2A32
:103700002A2A2A002020537461636B696E67206542
:1037100072726F7200202050726563697365206455
:1037200061746120627573206572726F720020206F
:103730004246415220416464726573733A20307886
:103740002578002020496D70726563697365206477
:1037500061746120627573206572726F720020203F
:10376000496E737472756374696F6E20627573202D
:103770006572726F7200457863657074696F6E2050
:103780006F6363757272656420696E20536563753B
:103790007265205374617465002A2A2A2A2A2048F7
:1037A000415244204641554C54202A2A2A2A2A00B4
:1037B0002020427573206661756C74206F6E2076D0
:1037C0006563746F72207461626C652072656164F8
:1037D0000020204661756C7420657363616C6174B0
:1037E000696F6E20287365652062656C6F772900AC
:1037F0002A2A2A2A2A204465627567206D6F6E691D
:10380000746F7220657863657074696F6E20286EBE
:103810006F7420696D706C656D656E7465642920C8
:103820002A2A2A2A2A005265736572766564204521
:103830007863657074696F6E2028005370757269C3
:103840006F757320696E7465727275707420284983
:10385000525120002A2A2A2A2A2025732025642949
:10386000202A2A2A2A2A006D7075004661696C6533
:103870006420746F20616C6C6F63617465206E6589
:1038800077204D505520726567696F6E2025750A47
:1038900000506172746974696F6E2025753A2073E7
:1038A000616E69747920636865636B206661696C19
:1038B00065642E00496E76616C696420756E64657E
:1038C000726C79696E6720726567696F6E20696EC8
:1038D00064657820257500464C4153485F3000539D
:1038E00052414D5F3000626F6172645F6E6F6E7344
:1038F0006563757265004750494F5F3000693263F8
:10390000004661696C656420746F20696E69746932
:10391000616C697A65206465766963653A20257310
:1039200000756E737570706F727465642073706566
:10393000656400636F6E6361742D627566206F76D7
:103940006572666C6F773A202575202B20257520CF
:103950003E202575004572726F72206F6E204932CD
:1039600043206C696E65206F6363757272656420B5
:10397000666F72206D65737361676520256400450D
:1039800072726F72202564206F6363757272656452
:1039900020666F72206D6573736167652025640012
:1039A0004932435F32006932635F6E7266785F74DA
:1039B00077696D00496E636F6D70617469626C65E3
:1039C00020706572696F642E005072657363616C5C
:1039D000657220666F7220706572696F645F6379CB
:1039E000636C6573202575206E6F7420666F756E2D
:1039F000642E0025733A2070696E2025752C207086
:103A0000756C73652025752C20706572696F642054
:103A100025752C207072657363616C65723A202580
:103A2000752E0050574D2070696E202564206E6FF2
:103A30007420656E61626C6564207468726F75676E
:103A4000682044545320636F6E66696775726174B1
:103A5000696F6E2E0050574D5F330050574D5F32E7
:103A60000050574D5F310070776D5F6E7266780061
:103A700070776D5F6E7266785F70696E5F73657484
:103A800000536C617665206D6F6465206973206EEC
:103A90006F7420737570706F72746564206F6E2020
:103AA0002573004C6F6F706261636B206D6F64658E
:103AB000206973206E6F7420737570706F727465F7
:103AC00064004F6E6C792073696E676C65206C6959
:103AD0006E65206D6F646520697320737570706FFB
:103AE0007274656400576F72642073697A6573201D
:103AF0006F74686572207468616E20382062697422
:103B00007320617265206E6F7420737570706F72B0
:103B1000746564004672657175656E6369657320CE
:103B20006C6F776572207468616E20313235206B5E
:103B3000487A20617265206E6F7420737570706FA3
:103B40007274656400435320636F6E74726F6C20EF
:103B5000696E6869626974656420286E6F204750D9
:103B6000494F206465766963652900557064617406
:103B70006520657863656564732063757272656E30
:103B80007420627566666572005350495F33007336
:103B900070695F6E7266785F7370696D0046616907
:103BA0006C656420746F20616C6C6F636174652058
:103BB000505049204368616E6E656C005541525407
:103BC0005F3100756172745F6E7266785F756172E5
:103BD000746500526573657474696E6720737973D8
:103BE00074656D00666174616C5F6572726F7200FE
:103BF0004552524F523A2043616E6E6F7420667583
:103C00006C66696C6C204558545F41504920726560
:103C100071756573742E0D0A005741524E494E4717
:103C20003A204F7074696F6E616C204558545F4143
:103C300050492072657175657374206E6F742066CB
:103C4000756C66696C6C65642E0D0A00556E6B6E42
:103C50006F776E206572726F7200756E6B6E6F7724
:103C60006E003E3E3E205A4550485952204641542F
:103C7000414C204552524F522025643A2025732052
:103C80006F6E20435055202564004661756C74208A
:103C9000647572696E6720696E746572727570748E
:103CA0002068616E646C696E670A004375727265A4
:103CB0006E74207468726561643A2025702028252E
:103CC00073290043505520657863657074696F6E81
:103CD00000556E68616E646C656420696E7465720F
:103CE0007275707400537461636B206F76657266D1
:103CF0006C6F77004B65726E656C206F6F70730030
:103D00004B65726E656C2070616E6963006D6169F0
:103D10006E006F730076322E342E39392D6E637338
:103D200032002A2A2A20426F6F74696E67205A6512
:103D300070687972204F53206275696C6420257316
:103D4000202573202A2A2A0A0000000000C0000053
:103D5000211A0100AB1E0100552701000C000120B3
:103D60000C00012001000000010000001C000120E7
:103D70001C00012000000000010000000000000005
:103D80000000000000000000000000000000000033
:103D90000080008000800080000000000000000023
:103DA0000080008000800080000000000000000013
:103DB0000080008000800080000000000000000003
:103DC00000800080008000800000000000000000F3
:103DD0000000000084000120840001200000000099
:103DE0000100000094000120940001200000000068
:103DF00001000000000000000000000000000000C2
:103E000000000000000000000000000000000000B2
:103E100000000000000000000000000000000000A2
:103E20000000000000000000000000000000000092
:103E300000C20100000103000000000000000000BB
:103E40000000000040420F000001030000000000DD
:103E5000000000000090D0030801012008010120AB
:103E60005A3401001C310100083101001C040120FA
:103E7000BC3B0100B83201009C320100F00001207F
:103E80003C340100B03201009C320100DC00012012
:103E90007A34010000000000000000000000000073
:103EA000F6380100983101007431010098040120B6
:103EB000553A010048320100703201006C000120C7
:103EC0005B3A010020320100703201005C000120E9
:103ED000613A0100F8310100703201004C0001200C
:103EE0000B330100D0310100703201003C00012091
:103EF000A0390100B8310100A43101000C000120FB
:103F0000893B010078320100943201007C000120DD
:043F100000000000AD
:103F1400C4010120C40101200000000001000000D0
:040000030000E25DBA
:00000001FF
